:020000040800F2
:10000000901000208D800008957F0008977F0008E1
:10001000997F00089B7F00089D7F0008A58000084D
:100020000000000000000000000000009F7F0008AA
:10003000A17F000800000000A37F0008A57F000842
:10004000A9800008AD800008B1800008B5800008D4
:10005000B9800008BD800008C1800008C580000884
:10006000C9800008CD800008D1800008D580000834
:10007000D9800008DD800008E1800008E5800008E4
:10008000E9800008ED800008F1800008F580000894
:10009000F9800008FD800008018100080581000842
:1000A000098100080D8100081181000815810008F0
:1000B000198100081D8100082181000825810008A0
:1000C000298100082D810008318100083581000850
:1000D000398100083D810008418100084581000800
:1000E000498100084D8100085181000855810008B0
:1000F000598100085D810008A97F0008618100081E
:1001000065810008698100086D810008718100081F
:100110007581000800000000798100087D810008D9
:1001200000000000818100088581000889810008A5
:100130008D8100089181000895810008998100084F
:100140009D810008A1810008A5810008A9810008FF
:10015000B57F0008AD810008B181000840F02000A3
:1001600070472DE9F14FB0B0924604910DF1420174
:100170003A9A2B9199464A7000200AE01AF8011B1E
:100180000498309A90470028049000F041860D981A
:10019000401C0D909AF8000050B12528EED10021A6
:1001A00000220791089209910A920B910C9204E0A7
:1001B0000D9800F02FBE41F001011AF8010F202820
:1001C000F9D023280CD02B2804D02D2805D0302896
:1001D00009D00BE041F00201EFE741F00401ECE748
:1001E00041F00801E9E741F01001E6E72A280FD1C4
:1001F000D9F8002052F8040BC9F8002000280F900D
:1002000003D540420F9041F004010AF1010A14E0C5
:100210000F92DFF8083C0AE00F98984205DA00EBED
:10022000800402EB4402303A0F920AF1010A9AF874
:100230000020A2F130000A28EED39AF800002E2800
:1002400003D04FF0FF320E9229E01AF8010F2A284E
:1002500009D1D9F8000050F8042BC9F800000E921B
:100260000AF1010A1BE02D280CBF0AF1010A002047
:1002700000220E92DFF8A44B0BE040B90E9AA24286
:1002800005DA02EB820503EB4503303B0E930AF1DE
:10029000010A9AF80030A3F130020A2AEDD3ADF832
:1002A00040100FF67C309AF8001000F0FBFE08B109
:1002B0001AF8010B8DF842009DF84200682805D11C
:1002C0009AF8000068280CD1622106E06C2804BF6F
:1002D0009AF800006C2804D171218DF842100AF1BF
:1002E000010A12A806901AF801BBBBF125012CD017
:1002F0001C3900F09481091F022940F290811339C2
:1003000000F0B884093900F08A81891E00F04D851B
:10031000491E00F0FA84491E022940F28081091F1B
:1003200000F0F384491F00F0EF80491E00F0A28422
:10033000491E00F0D780C91E0CD0891E00F09A8497
:10034000C91E00F0978400F03BBD012307932521CF
:1003500000F033BDD9F8000050F8044BC9F8000094
:10036000002C059440F0AB802B994878002800F0D1
:10037000A1804FF0FF340FF6B02000F0ADFE241A3C
:1003800040F0468500F028BD01236A4602A93046A8
:1003900000F00EFE002840F03B85641EF4D130963C
:1003A000079C12AF74B1309E17F8011B0498B04738
:1003B0000028049000F02C850D98401C641E0D90C0
:1003C000F2D130960A9C3021002C8DF800100CDD03
:1003D000309E01236A4602A9304600F0E9FD00285C
:1003E00040F01685641EF4D13096059F089C74B1C8
:1003F000309E17F8011B0498B0470028049000F0C5
:1004000007850D98401C641E0D90F2D130960B9C10
:100410003021002C8DF800100CDD309E01236A463F
:1004200002A9304600F0C4FD002840F0F184641EAB
:10043000F4D1309605980899099C471874B1309EFC
:1004400017F8011B0498B0470028049000F0E084DE
:100450000D98401C641E0D90F2D130960C9C3021FA
:10046000002C8DF800100CDD309E01236A4602A995
:10047000304600F09DFD002840F0CA84641EF4D18F
:1004800030969DF8400041077FF584AE2020002D76
:100490008DF800007FF77EAE309C01236A4602A9EA
:1004A000204600F085FD002840F0B2846D1EF4D196
:1004B00030946FE60FF65830059000F08DBC0E9D1D
:1004C000002D04D5204600F027FE044607E02A460A
:1004D000204600F02BFE002814BF041B2C46089475
:1004E00000F07ABCD9F8001051F8040BC9F80010DC
:1004F00020F00004002121F0FF35CDE9024512ABC8
:100500000593782100F04DBC2B99487820B14FF02D
:10051000FF340FF6CC2030E79DF84200622860D00F
:10052000682817D06A283FD06C2806D0712847D099
:1005300074282CD07A281DD062E0D9F8001051F828
:10054000040BC9F80010002866D14FF0FF340FF6F5
:10055000A82012E7D9F8001051F8040BC9F80010D0
:1005600020B94FF0FF340FF6902006E70D99018077
:1005700000F032BCD9F8001051F8040BC9F8001093
:10058000002849D14FF0FF340FF66C20F5E6D9F87A
:10059000001051F8040BC9F8001000283CD14FF0AE
:1005A000FF340FF65420E8E6D9F8001051F8040B98
:1005B000C9F8001080B94FF0FF340FF63C20DCE69C
:1005C000D9F8001051F8040BC9F8001020B94FF009
:1005D000FF340FF62420D0E60D9AD317C0E900238C
:1005E000FAE3D9F8001051F8040BC9F8001020B94B
:1005F0004FF0FF340FF60020BFE60D990170EBE3DA
:10060000D9F8001051F8040BC9F8001020B94FF0C8
:10061000FF340FF6E410B0E60D990160DCE39DF8BD
:1006200042004C2807BFD9F80010CA1DD9F80000B5
:10063000C21D22F00702C9F80020D2E900010832E9
:10064000C9F80020CDE90201C80F02D007982D217A
:100650000AE0BDF84000810702D507982B2103E08E
:10066000C00705D50798202112AA1154401C0790F5
:1006700012A807994BF0200300EB010CDDE9020101
:10068000CDE92C01612BCDF814C021AC0BD00E9814
:10069000002848BF062105D404BF4BF0200067287E
:1006A00001D101210E91DDE902014F0047EAD07727
:1006B0007E15FF174FF0FF32974208BF964210D1C8
:1006C000090341EA10510003002908BF002808D09F
:1006D000ABF1610503211A2D089118D30FF63811DB
:1006E00010E0DDE902014A00521512F1010F11D1AB
:1006F00008030FD1ABF1610503211A2D08911FD317
:100700000FF61C110322604600F03CFD64E30FF677
:100710000411F7E7DDE902016A4600F03FFDCDE98B
:1007200002014BF02000612811D1059830210170A1
:10073000821C0592BBF1610F0CBF7821582102E0A9
:100740000FF6D801DEE741700798801C0790DDE9BD
:10075000020120F0000231F0004308BF002A02D15C
:100760000026002542E14BF02008B8F1610F40F06F
:1007700092800E98002847BF21210191401C0190D2
:10078000019FDDE92C017F1C00220023DDE90245E9
:1007900000F03CFD38BF85F0004500998DF88420BD
:1007A000091F002F00910DF1850632DD20462946F4
:1007B0000022002300F044FD2BD21C2200F05AFD41
:1007C00004460D4600F000FEFF1F002F804609DDA5
:1007D00000F01AFE02460B462046294600F0E4FED1
:1007E00004460D46F01D0721B8F1000F0CDD491E2F
:1007F0005EBF08F00F0200F8012D4FEA2818F3D56C
:1008000002E0002200F8012D491EFAD5C61D002F76
:10081000CCDC0DF18500361A01980DF18504864275
:10082000D8BF304600282FD4B04206DA0DF185013A
:100830000A5C082AA8BF0F2100DA0021024621AB7A
:10084000134400E0401E13F80159521E8D42F9D0A6
:100850000F2904D10DF185018B5C5B1C8B54002AA0
:1008600004D50099091D21AC401C0091411E0BD4F8
:10087000621813783033DDB23A2DA4BF5B443A3BA3
:10088000491E02F80139F4D50E99002940F1AC80D7
:10089000421E0E92A8E00099DFF8042747F2975015
:1008A000414391FBF2F20092DDE92C45C2F10702CF
:1008B000002A25F0004504DD2046294600F04CFBC7
:1008C0000BE052420020DFF8DC1600F045FB024648
:1008D0000B462046294600F0D9FE04460D46B8F1E5
:1008E000660F06BF009F0A3706270E983F18142F81
:1008F000C8BF142730208DF884000DF18506002F25
:1009000034DD2046294600F0E5FF01460A4606F19F
:10091000080304200A26B2FBF6F606EB860EA2EBCD
:100920004E02303203F8012C0A22B6FBF2F202EB3F
:10093000820EA6EB4E063036401E03F8026DE9D15A
:10094000083F002F03F10806D9DD084600F0D4FF68
:1009500002460B462046294600F026FE0022DFF81C
:10096000483600F0D7FF04460D46CAE70DF1850072
:10097000361A0DF1850404E00098401E761E0090A2
:10098000641C20783028F7D0B8F1660F02D10098A7
:10099000401C04E0B8F1650F0CBF012000200E9947
:1009A00040188642B8BF701E00281DD4B04204DA39
:1009B000215C3429C8BF392100DC30210246631E86
:1009C0009D1800E0401E15F80169521E8E42F9D0B4
:1009D000392902D1A15C491CA154002A04D50099EF
:1009E000491C1C46401C00910646009D01F088F8F9
:1009F000406A0778DDF8388030B2002802DC012632
:100A00000FF220644BF02000662808BF6D1C16D042
:100A1000672845D128B210F1040F47DB404545DA7D
:100A20009DF840006D1C010703D430B24045D8BF8B
:100A3000804628B2B8EB000848BF4FF000080FFA14
:100A400085FBBBF1000F00F3B4800898411C0891AE
:100A5000302205990A54B8F1000F03DC9DF84000DC
:100A6000010704D50898411C089105990F5418EB0B
:100A70000B0FB8BFC8F100052DB26842454432B231
:100A80000B909542B8BF2E46059B089836B2099642
:100A900032462146184400F075FBAD1B0C95D2E0A0
:100AA000BBF1610F17D14FF0700B19E030B2404528
:100AB00004DA9DF840100A0758BF8046B8F10108D3
:100AC00048BF4FF00008BBF1670F14BF4FF0450B54
:100AD0004FF0650B04E0BBF1410F08BF4FF0500B26
:100AE0000898411C0891B8F1000F059914F8012BE2
:100AF0000A5403DC9DF8400001071AD50898411CF0
:100B00000891B8F1000F05990F5412DD761E30B22E
:100B10008045B8BF46460598089B32B22146184426
:100B200000F030FB089936B271180891A8EB060066
:100B30000B9005980899084429B2002980F800B064
:100B400003D42B224270821C04E02D2242700D46F9
:100B5000821C6D4200212CAB28460AE004460A2084
:100B600094FBF0F000EB8005A4EB450403F8014B87
:100B7000491C00B20028F1DC012906DC4BF0200002
:100B8000652804BF302002F8010B00292CAB08D1E6
:100B9000302002F8010B06E0491E585C303002F8A4
:100BA000010B0029F8DC059908980844121A0992EB
:100BB00049E030B229B288421CDA0598089B32B26B
:100BC0002146184400F0DEFA089936B271180891EF
:100BD000ABEB0600B8F1000F0B9003DC9DF8400072
:100BE000020704D5059847540999491C0991CDF885
:100BF000308028E00598089B2AB22146184400F06E
:100C0000C1FA0898761B5844B8F1000F089003DC2D
:100C10009DF840100A0703D5411C089105990F540F
:100C200030B28045B8BF46460598089B32B204EB07
:100C30000B01184400F0A6FA089836B23018089054
:100C4000A8EB06000B909DF8400000F0140010285F
:100C500040F0C280079A08980B99821809988A1860
:100C600082180C980F998018884280F2B580081A73
:100C70000A90B1E09DF84200622808D068280ED0A2
:100C80006A2814D06C281FD0712810D01CE0D9F825
:100C9000001051F8040BC9F80010C0B21AE0D9F8DE
:100CA000001051F8040BC9F8001080B212E0D9F816
:100CB0000000C21D22F00702C9F80020D2E900019D
:100CC0000832C9F8002006E0D9F8001051F8040BEA
:100CD000C9F800100021CDE902019DF8400001078C
:100CE0005AD5DDE90223002B08BF002A54D04BF06F
:100CF0002000782850D1079812A930220A54401CAD
:100D0000431C079301F800B046E09DF842006228BA
:100D100008D068280ED06A2814D06C281FD07128FB
:100D200010D01CE0D9F8001051F8040BC9F80010DD
:100D300040B21AE0D9F8001051F8040BC9F80010BD
:100D400000B212E0D9F80000C21D22F00702C9F873
:100D50000020D2E900010832C9F8002006E0D9F8E5
:100D6000001051F8040BC9F80010C117CDE90201B9
:100D7000002902D507982D210AE0BDF8400081071F
:100D800002D507982B2103E0C00705D5079820213D
:100D900012AA1154401C079012A80799014405910A
:100DA000594602A800F04EF816E001200790D9F845
:100DB000000050F8041BC9F800008DF848100BE043
:100DC00001212522BBF1000F07918DF8482003D0A7
:100DD000022207928DF849B00F9D07990A986D1A63
:100DE00008992D1A0B986D1A09992D1A0C986D1ADD
:100DF0009DF840102D1A48073FF5D2AA2021002D5A
:100E00008DF800107FF7CCAA309E2C46FFF7BCBAB5
:100E10004FF0FF3031B0BDE8F08F0000CBCCCC0CF0
:100E2000686A6C747A4C00007072696E74665F73E5
:100E30003A2062616420257320617267756D656E6A
:100E4000740000002DE9FC4707468A463C6950467D
:100E50006F2808BF082505D0FFF780F9782814BF50
:100E60000A251025D7E900013C2680468946BAF1BB
:100E7000640F18BFBAF1690F05D1002903D5D8F165
:100E8000000869EB4909B9F1000F08BFB8F1000F7C
:100E90000CD1386B50B9082D3AD197F838000107BA
:100EA00036D530223B2684F83B2031E08DF800A077
:100EB000404649462A46EB1700F028FE3032D0B2B1
:100EC000761E3A2801960EDAA255404649462A4631
:100ED000EB1700F01BFE80465FEA010908BFB8F17E
:100EE000000F05D108E09DF800001218513AEBE719
:100EF000F868A1198842DBD3082D09D197F838008A
:100F0000010705D5A05D302802D0761E3020A055FF
:100F1000C6F13C03BB61A119F960386B834208DA62
:100F2000C31A3B624FF6EF70398F01403987BDE835
:100F3000F38700280ED597F8380000F01400102829
:100F400008D17A6B7969386A521A121AD21A002AB1
:100F5000C8BF3A62BDE8F3872DE9D04306460F4685
:100F600014464FF00008DFF8449012E0E00707D580
:100F700042464B463046394600F0CCFC06460F460A
:100F80004046494642464B4600F0C4FC6410804649
:100F90008946002CEAD130463946BDE8D0830000AE
:100FA000A08601000000F03F84D797410000244054
:100FB000F8B505460E4617461C4600205CB117F8EA
:100FC000011BB068A847B06030B1F06A401CF06205
:100FD0000020641EF3D1F2BD4FF0FF30F2BD0000DF
:100FE0007072696E74665F733A20256E206469734F
:100FF000616C6C6F776564007072696E74663A201C
:1010000062616420256E20617267756D656E740083
:10101000000000006E616E004E414E00696E660079
:10102000494E46003000F0B4024610689568131827
:10103000506803EB5004C00748BF4D44A3422DD075
:1010400013F8016B16F0030004BF13F8010BC01C6A
:1010500031090F2907D113F8011B0F3103E013F8F1
:10106000017B05F8017B401EF9D10029E6D013F879
:10107000010BC6F38106032E08BF13F8016B00EBCA
:101080000620404228440026B71E8F421EBF10F89B
:10109000017B05F8017B761CF6D1CFE7F0BC02F1AD
:1010A0000C007047C9B202788A421AB11CBF10F80E
:1010B000012FF9E718BF0020704703681AB95A1EBC
:1010C000026008467047197811B94FF0FF30704739
:1010D000591C01601878704780B500B906A0054911
:1010E0000B681BB122220021984701E000F091FD1E
:1010F000222002BD8C0C0020636F6E7374726169D4
:101100006E742068616E646C65723A20626164205E
:101110006D6573736167650000F1010310F8011BD1
:1011200011B110F8011BFBE7C01A7047C9B2830761
:1011300006D0521E22D310F8013B9942F7D11FE08E
:10114000083A13D302F1040241EA012141EA0141C4
:1011500050F8043B121F21BF4B40A3F1013C2CEA85
:10116000030C1CF0803FF3D0C9B2001F083210F806
:10117000013B521E28BF91EA030FF8D818BF012087
:10118000401E70474AB1000011F8013B521E00F8A2
:10119000013B1CBF11F8013BF8E7704710B514463E
:1011A00000F002F8226010BDC1F30A5343B14A00B7
:1011B00012F5001F28D2A3F2FE32A1EB02517047B4
:1011C00050EA410C20D001F0004C31EA0C01B1FA98
:1011D00081F204BFB0FA80F3D2180B3AB2F12003C7
:1011E0002CBF00FA03F1914041EA0C013EBFC2F16D
:1011F000200C20FA0CF319439040524240F2FD3388
:10120000D21A01EB035170470022704741EA030CE8
:1012100050EA4C0C52EA0C0C4FF4001C09D307D0D6
:101220001CEB410F9CBF1CEB430F8B4208BF82425B
:1012300070471CEB430FFBD8994208BF90427047A0
:1012400041EA030C50EA4C0C52EA0C0C4FF4001C1F
:1012500009D307D01CEB410F9CBF1CEB430F9942F5
:1012600008BF904270471CEB410FFBD88B4208BF70
:1012700082427047124254D440F2FF7C1CEA115360
:101280000FD0634531D09B1863453CBF01EB025141
:10129000704701F0004141EA0C510020AFF300809B
:1012A000704750EA410320D001F0004C91EA0C0154
:1012B0001CD0B1FA81F30B3B9A420DD9D21A994056
:1012C00051EA0C01C3F1200C20FA0CFC6144984057
:1012D000531C40F2FF7CD7E7914041EA0C01C2F178
:1012E000200C20FA0CF3194390407047B0FA80F3B9
:1012F0001533202BE0D3202AEED3203A203B9A420C
:1013000009D9D21A00FA03F141EA0C010020531C5A
:1013100040F2FF7CB8E700FA02F141EA0C0100203C
:101320007047524240F2FF7C1CEA11530DD06345D6
:10133000DBD0B2EB030C3CBFA1EB025170470CF1C8
:10134000010221EA035141F4801150EA410CCCD052
:1013500001F0004C352A27DC30B481EA0C01B2F1EF
:10136000200309DAC2F12003044601FA03F5D04054
:101370002843D1409C400CE0C3F12002450020FAF4
:1013800003F418BF44F0010421FA03F091400C4328
:10139000002174F1004550F1000051EB0C01244292
:1013A00030BC7FF47BAF70476146002076E78268EF
:1013B000521C8260426832B10268531C0360117093
:1013C0004168491E41607047C1F30A5340F21E4212
:1013D000D31A0CDDCA0283F3070342EA505242F0EB
:1013E0000042DA4002EBE17282EAE17070476FEA94
:1013F000E17203F2E13008B182F000407047026808
:10140000531C03601170704710F0004160B148BF79
:101410004042B0FA80F29040D21CC2F5846241EAA8
:10142000025202EBD021400570472E0070B491EAC1
:10143000030F4FF0004540F1BF806B40841A71EB01
:10144000030604D26E40001BB141121973414FF4E0
:10145000001C1CEB410F34BF7CEB430683E00C0DFA
:10146000A4EB1356362E00F37C80012E45EAC323ED
:1014700041DC43EA525312BFD20292025B082405B8
:1014800045EAC12141EA5051D2EBC020994125D40F
:1014900007D1B0FA80F610FA06F162D000202036AB
:1014A00008E0B1FA81F6B140C6F1200220FA02F25A
:1014B0001143B0404FEAF474B4EB465434F00106E3
:1014C0004FEA74040AD8D6F50016760D04F00044ED
:1014D000F04061FA06F25040F1404840C00A40EA4C
:1014E000415021F0004128BF5FEA500550F1000053
:1014F00044EBD12135E0DB0A45EAC121C90AB6F146
:1015000020050EDD42EA0242120CC5F1200603FA64
:1015100006F6EB4042EA06056D42984161F1000192
:101520000DE062FA06F5F240554063FA06FC82EAE5
:101530000C02F3405A406D42904161EB030111F4FB
:10154000801F05D1641E620502D06D0040414941F3
:1015500021F48011430875F1004350F1000041EB84
:10156000045170BC70471CEB410F15D223F00043AF
:1015700052EA43060BD04FEA4C0CBCEB410F04D8A7
:101580000C0D661E342EB7DDEBE7801A994150EA48
:10159000410608BF0021E4E708BF1CEB430F28BF4A
:1015A0006FF00001DDE7000070B491EA030F4FF027
:1015B00000457FF543AF6B40841A71EB030603D2FD
:1015C000001BB141121973414FF4001C1CEB410F79
:1015D00034BF7CEB430442E00C0DA4EB1356352ED4
:1015E0004FDC45EAC323DB0A45EAC121C912B6F143
:1015F00020050DDD63FA05F6EB4086EA030512428D
:1016000018BF45F00105C01851F100010CD213E0DC
:1016100062FA06F5F2405540F3415A40B340F340B8
:101620005A408018594107D349085FEA30005FEA01
:10163000350528BF45F0010501F58011420875F117
:10164000004250F1000041EB04514E0016F5001F1E
:1016500070BC38BF70470020090D090570471CEBAE
:10166000410F10D252EA43060BD0BCEB410F05D814
:101670000C0DAB43661E342EB6DD02E0AB43801882
:10168000594170BC704770BC70474300F0B540F2E0
:10169000FF7581EA030C0CF0004C15EA11541DBFD4
:1016A00015EA1357AC42AF42E5E0BC41C1F3130168
:1016B000C3F31303801A994143F4801304D2641EC8
:1016C0000018494180185941C90241EA5051B1FB03
:1016D000F3F603FB1611A2FB0675D7EBC020A94158
:1016E00002D2761E80185941C90241EA5051B1FB1D
:1016F000F3FE03FB1E11A2FB0E75D7EBC020A94120
:1017000003D2AEF1010E80185941890241EA90518D
:10171000760546EA8E2EB1FBF3F603FB1611A2FB0B
:101720000675D7EB8020A94102D2761E8018594158
:10173000C90241EA50514EEA060EB1FBF3F603FB33
:101740001611A2FB0675D7EBC020A94102D2761E66
:1017500080185941C90241EA5051B1FBF3F703FB2C
:101760001711A2FB0735D3EBC020A94167F1000791
:101770000CBF004247F0010766F3D5274FEA1E3140
:10178000B80814F5806412DDBD0775F1004250EB16
:101790000E5051EB045111F5801F5CBF41EA0C0162
:1017A000F0BD4CF07F6141F0E0410020F0BDBD078D
:1017B0006D0840EA0E5041F48011D4F10104B4F1F7
:1017C00020060ADAC4F120060200E04001FA06F31E
:1017D000E1401843B24015430EE0342C13DCC6F14F
:1017E000200445EA40056D0820FA06F2154321FA67
:1017F00006F0A1400D43002175F1004250F10000B8
:1018000051EB0C01F0BD00205FEA0C01F0BDCFB937
:1018100092185B41B3FA83F704BFB2FA82F6BF199C
:101820000B3FB7F120062FBF02FA06F3BB40C7F10A
:10183000200622FA06F638BF3343BA401CB1E41939
:10184000641E33E77F4231F00041B1FA81F404BFF6
:10185000B0FA80F6A4190B3CB4F120062FBF00FAB1
:1018600006F1A140C4F1200620FA06F638BF314344
:10187000A0403C1B1AE7AC421ABF05EA1357AF421F
:1018800012E050EA41061CBF52EA4306BFE750EAA5
:101890004107304661461CBF41EA0551F0BD52EA9E
:1018A000430C08BFC143F0BD00204FF4001616EBF7
:1018B000410F98BF16EB430F08BF16EB410F24BF33
:1018C000C14305E016EB430F0CBF61464CEA0551DE
:1018D000F0BD0000400D40F21E4C40EAC120BCEBC0
:1018E000115C40F0004003D48CF30701C8407047FE
:1018F0006FEAE1707047000050B1B0FA80F18840A3
:10190000C91CC1F58461090501EBD0214005704770
:101910000146704730B540F2FF7C1CEA11541DBFF0
:101920001CEA1355644565453FE0641981EA030CE0
:101930006FF35F530CF0004C43F48013C90241F085
:10194000004141EA505EC5021100A5FB02020028D9
:101950004FF00000EEFB01204FF00001E3FB0521FA
:1019600018BF42F00102401800214941E3FB0E017B
:10197000A4F580640D0302D292184041494154F10C
:10198000010470DD450872F1004250F1000051EB96
:101990000451A1F5801102D441EA0C0130BD40F29E
:1019A000FF7E4CEA0E51002030BD0CEA1355644511
:1019B00018BF654581EA030C0CF0004C41D050EA99
:1019C000410E1CBF52EA430E02E06146002030BDCA
:1019D00024422C441BD15FEA050EF6D0090302BF56
:1019E00001460020AEF1140EB1FA81F5AEEB05040C
:1019F00001FA05FE0C35C5F1200100FA05F5C840D5
:101A00004EEA000E6FF35F5343F480139CE733F00C
:101A10000043B3FA83F504BFB2FA82FE75440B3D6E
:101A2000641BB5F1200E2FBF02FA0EF3AB40C5F1D7
:101A3000200E22FA0EFE38BF43EA0E03AA40641CB1
:101A40007CE750EA410E14BF52EA430E6FF00001EA
:101A50004FF4001515EB430F8EBF194615EB410FE0
:101A60009DE7B4D830BDD4F10104B4F120050FDAFC
:101A7000C4F12005520828BF42F0010210FA05FE09
:101A800001FA05F57244E2BFE0402843E1400FE06F
:101A9000352C9ADCC5F1200452EA400220FA05F206
:101AA00018BF42F0010231FA05F0A1400A430021BB
:101AB00072F1004250F1000051EB0C0130BD00000A
:101AC000613807E005E0A0F161011A2901D2012087
:101AD000704741381A288041C00F7047A0F10901B2
:101AE000052901D3202801D101207047002070472B
:101AF000A0F141011A2938BF2030704701487047D2
:101B0000014870474800002010000020D3BBD9B125
:101B1000B2F5803F5BD2022A1ED98C46B1FBF2F1AE
:101B200002FB11C31B0443EA1043B3FBF2FC02FBAC
:101B30001C3380B240EA0343B3FBF2F002FB1032E5
:101B400040EA0C4000237047022A05D98446B0FBC6
:101B5000F2F002FB10C270474AB105D100F0010259
:101B600049085FEA3000704700220023704700F008
:101B700053B80B000200002100207047F7D3002269
:101B800000237047904271EB030CF2D370B5B1FAA9
:101B900081F4B3FA83F52C1BA340C4F1200532FA7B
:101BA00005F63343A2405FF00046E64002E05B08E2
:101BB0005FEA3202841A71EB030524BF20462946EE
:101BC0007641F4D302000B003000002170BD70B5E7
:101BD000B1FA81F4B2FA82F5C4F120046419B4F1C7
:101BE0002006DAD3B2405FF00044F440002502E062
:101BF00052085FEA3303C61A71EB020E24BF304667
:101C0000714664416D41F3D302000B0020002900AE
:101C100070BD012000F002B87047000080B5AFF33E
:101C20000080024A11001820ABBEFBE7260002002C
:101C300038B5040001D1012032BD04F18405686883
:101C400008B900F017F800F01AF808B100F031F800
:101C500000F02CF8012804D000F004F821F02A014B
:101C600016E032BD2068416821F49041416020684F
:101C70008168704700212970204600F082BF24202F
:101C8000686020680168490849000160A06A7047DF
:101C9000816000F004F8BDE8324000F0AFBB20687E
:101CA000016841F00101016020467047204600F0C4
:101CB0002DBA204600F03FBB38B5040001D1012009
:101CC00032BD04F184052420686000F014F8226815
:101CD0000020002110602368596021688860204638
:101CE00000F0E0FF0020E86000216960A860E16684
:101CF0002067297032BD20680168490849000160E9
:101D000070472DE9F843054605F15406706B0C4603
:101D10001746994620283ED10CB1380001D1012048
:101D20003AE00020F0632121716301F06DF8378003
:101D300080467780A868B0F5805F04BF28690028D6
:101D40001ABF204600272746044611E000228021C2
:101D500000F024F8D8B92868002C12BF14F8011B31
:101D600037F8021BC1F3080181627088411E71803F
:101D70007088CDF8009043460028E7D1002240212A
:101D800000F00CF818B920207063002004E0202037
:101D90007063032000E00220BDE8F283284600F0D3
:101DA00074BB38B50346D3F88C0020280AD109B19A
:101DB000100001D1012032BD00F006F8BDE8384026
:101DC00000F0ABBB022032BD0020D8661868DFF8F7
:101DD0003843A0420CD04068040209D5186850E886
:101DE000004F054644F0806445E800400028F5D1E6
:101DF0001846704728688168480670472DE9F04109
:101E000005462A68D36940F60F0610460768D2F8DF
:101E1000088005F15C0407F0200003F02001334244
:101E20000ED1002914D018B95FEAC80040F18780AC
:101E3000A169002900F02F812846BDE8F04108473C
:101E4000DFF838C818EA0C0F04BFDFF834683742EF
:101E500075D0DE0709D5FE0507D54FF0010EC2F893
:101E600020E0626B42F0010262639A0748BF5FEABA
:101E7000C87206D52E6802223262626B42F00402FA
:101E800062635A0748BF5FEAC87206D52E6804220B
:101E90003262626B42F0020262631A070DD50028BB
:101EA00008BF18EA0C0F08D0D5F800C00822CCF8FB
:101EB0002020626B42F0080262631A0509D57B019B
:101EC00007D52F684FF400623A62626B42F020023D
:101ED0006263626B002A31D039B110B95FEAC80081
:101EE00003D5A16909B128468847606B29688A68CB
:101EF000510602D410F0280F1BD000F0D4F8FFF7E1
:101F000079FF11D500F0D2F8FCD1606A60B10FF210
:101F1000A171C166606A00F0BBFF00280ED0606A44
:101F2000C16EBDE8F04108472846BDE8F04100F029
:101F3000D0BF284600F0CDFF00206063ABE02069F1
:101F4000012875D1D80673D5F90671D51020106215
:101F50002A6821889068420632D5626A1068806CCF
:101F600080B2002823D0884221DA6080106D812859
:101F700016D000F0B4FCFCD100F0B8F8FCD100F0B1
:101F8000A8F8FCD1202020630021216100F09CF8FA
:101F900021F0100100F083F8F8D1606A00F03AFFF8
:101FA0000220606121886088091A89B206E08842AF
:101FB00004BF106D81286ED102226261284633E091
:101FC00062886088891A00281CBF88B2002862D005
:101FD0002A46106850E8003F054623F4907345E810
:101FE00000300028F5D1106800F1080353E8003FE5
:101FF00000F10808DFF82C03034048E8003000280F
:10200000F1D12020206300232361A361136853E8EA
:10201000003F156823F0100345E800300028F5D193
:102020000220606189B21046BDE8F04100F052BF65
:1020300018060AD5390658BF5FEA082005D5E169B8
:1020400049B32846BDE8F0410847580611D579063E
:102050000FD500F039F821F0400100F020F8F8D158
:102060002020E0620021E1612846BDE8F04100F057
:1020700032BF180206D5790004D52846BDE8F041E4
:1020800000F02ABFD80148BF002F04D52846BDE87C
:10209000F04100F022BFBDE8F08141F4807142E8D8
:1020A000001000287047284600F0BDBA296801F1E9
:1020B000080252E8001F286800F1080321F04001DF
:1020C00043E8001000287047286850E8001F0246C7
:1020D0007047286800F1080151E8001F00F108036B
:1020E00021F0400143E8001000287047286800F103
:1020F000080151E8001F00F108034908490043E8BE
:10210000001000287047000000240046F8B504467F
:102110002268DFF8F40600251368A16803402069EF
:102120000B4361690343E0690B4303431360516848
:10213000E06821F4405101435160DFF88417A3693E
:102140008A421CBF206A03439668DFF87807DFF8ED
:1021500078E7064033439360D36A606A0FF25C56B7
:102160001B0940EA0313DFF86407DFF86477D362E2
:102170004FF4004372453AD13F6807F00307032F3D
:102180005AD8DFE807F0025350564FF0010CE169CE
:102190004FF6F077B1F5004F40F09080BCF1000FA2
:1021A0000FD0BCF1010F00F08180BCF1040F0CD006
:1021B000BCF1080F00F07D80BCF1100F00F07C80B6
:1021C000A5E001F0ADF9002810D000F0ADF84A0804
:1021D00002EB4002B2FBF1F0A0F11001B942EFD2E4
:1021E0000740C0F3420007432068C76090E0DFF873
:1021F000A4C762450CD13F6817F00C0706D0042F26
:1022000014D0082F0FD00C2F13D015E0AC46BEE72A
:102210008A4211D1BF6807F00307032F0CD8DFE80B
:1022200007F01C0502084FF0040C07E04FF0080C03
:1022300004E04FF0100C01E04FF0200C8A42A6D1D0
:10224000BCF1020F09D0BCF1040F0AD0BCF1080F99
:1022500015D0BCF1100F15D059E001F06FF900282E
:1022600056D0616A36F81120B0FBF2F6626802EBD4
:1022700042018E424BD31303B34205D247E001F033
:1022800030F9ECE71846ECE75008002110EB062087
:10229000DFF8A87751EB16610023FFF737FCA0F5B4
:1022A0004076BE4233D22168C86031E001F03DF98A
:1022B00089E701F016F986E7184686E7BCF1000FBA
:1022C0000CD0BCF1010F1AD0BCF1040F09D0BCF145
:1022D000080F17D0BCF1100F17D018E001F020F94B
:1022E000B0B100F021F800EB5100B0FBF1F0A0F12B
:1022F0001001B9420BD2226880B2D06008E001F030
:1023000014F9EDE701F0EDF8EAE71846E9E70125F1
:1023100004F168000121002341800180C360036152
:102320002846F2BDFEFFFFEF626A616836F81230A0
:10233000B0FBF3F0704790F828100A0706D5026842
:102340005368816B23F400430B43536090F82810CB
:10235000CA0706D502685368C16A23F400330B43E9
:10236000536090F828108A0706D502685368016BFD
:1023700023F480330B43536090F828104A0706D5A6
:1023800002685368416B23F480230B43536090F839
:102390002810CA0606D502689368C16B23F48053DF
:1023A0000B43936090F828108A0606D5026893685C
:1023B000016C23F400530B43936090F828104A06F5
:1023C00010D502685368416C23F480130B435360AB
:1023D000436CB3F5801F05D15368816C23F4C003AF
:1023E0000B43536090F828100A0606D501684A6826
:1023F000C06C22F4002202434A607047F8B50546DB
:1024000005F184040020E06000F0FEFC0646286828
:102410006FF07E4701680A0711D500973346002206
:102420004FF40011FFF7BAFC48B1FFF74DFE21F061
:102430008001FFF734FEF8D12020606017E02868A3
:1024400001684A0717D50097334600224FF48001F0
:10245000FFF7A4FC78B1FFF737FE21F49071FFF786
:102460001EFEF8D1FFF742FEFCD12020A060002123
:1024700021700320F2BD202060602021A160002097
:10248000E866002129672070F2BD2DE9F04105467C
:102490000E4690461F46069C2868C1693140B142ED
:1024A0000CBF01200020404535D114F1010FF3D0BD
:1024B00000F0AAFCC01B844200D314B90320BDE87D
:1024C000F081286801684A07E6D5802E18BF402EA3
:1024D000E2D0C169080704D42968C8690105DBD5C1
:1024E0000CE02A6808201062FFF7DDFD05F184008A
:1024F0000821C160002202700120E0E729684FF442
:1025000000600862FFF7CFFD05F184002021C16063
:1025100000220270D2E70020D1E750B5034699654A
:1025200003F15C010A804A80002088619868FF24DA
:10253000B0F5805F04D1186990B940F2FF140FE044
:1025400018B9186960B17F2007E0B0F1805F06D14B
:10255000186908B97F2403E03F20888001E0002447
:102560008C800020486322240C63186800F098F8DF
:1025700044F0010446E800400028F6D18868B0F134
:10258000005F21D1888982421ED39A68B2F5805FAC
:1025900004BF1869002803D10FF259328A6109E09B
:1025A0000FF27D248C61186920B100F02FF8FFF73D
:1025B00074FDFAD100F02FF841F0805144E800108A
:1025C0000028F7D1002050BD9868B0F5805F04BFA7
:1025D000186900280CD10FF24D128A61186850E872
:1025E000001F024641F02001FFF759FDF6D1E9E74F
:1025F0000FF2E1028A6118690028EFD000F006F8B6
:1026000041F49071FFF74BFDF8D1DBE7196851E811
:10261000001F1A687047186800F1080151E8001F90
:1026200000F10804704710B500F00EF8FCD100F07E
:1026300015F8FCD1C16E00F025F82021C0F88C10EF
:102640000022C266426710BD016851E8002F0B46A8
:1026500022F4907243E8002100297047016801F1DB
:10266000080252E8002F01F10804DFF844140A4080
:1026700044E800210029704700000000010000101C
:1026800020010004012909D1026852E8002F0368E3
:1026900022F0100243E800210029F5D170471068AC
:1026A00000F1080454E8004F00F1080670470000EC
:1026B000C06D0021A0F85E1000F00BBC010002000C
:1026C0000400060008000A000C0010002000400072
:1026D0008000000138B500F04DF81ED14B6A91889A
:1026E000846D0B402370816D4B1C00F049F818D1AC
:1026F00000F04DF800F060F8FCD100F06AF80BD162
:102700000023136100F04EF8FCD10168CB69DC06B0
:1027100044BF10230B6279E07DE0886940F0080037
:10272000886131BD38B500F025F81ED14B6A91881B
:10273000846D0B402380816D8B1C00F021F818D133
:1027400000F025F800F038F8FCD100F042F80BD189
:102750000023136100F026F8FCD10168CB69DC0688
:1027600044BF10230B6251E055E0886940F0080037
:10277000886131BD00F15C020168136B222B704748
:10278000836551884B1E5380518800297047036828
:1027900053E8003F046823F4907344E800310029B3
:1027A000F5D17047016851E8003F0C4623F0100353
:1027B00044E8003100297047016801F1080353E83B
:1027C000003F01F108055B085B0045E80031002986
:1027D000704720211163002393610021516101683A
:1027E000374B99420CD049680B0209D5016851E872
:1027F000003F0C4623F0806344E800310029F5D106
:102800001169012970470000F369FFCF1188BDE805
:10281000344000F05FBBBDE8324000F0B3BA0000C6
:102820002DE9F84300F00CF946D1A089002835D0F5
:10283000B80633D500F0B0F80870A86D421C00F05F
:10284000D9F812D0F90748BF5FEAC85200F0AAF8D9
:1028500003D5F10701D500F0C5F800F0ACF820B1C0
:10286000284600F036FB0020606360880028DFD136
:1028700000F035F8FCD100F0D3F8FCD100F0FEF800
:1028800009D100F0EBF844BF1021016221882846ED
:1028900000F020FB02E0284600F074FA608868B17E
:1028A000A18988420ADA00F0AEF8FCD18148A06123
:1028B00000F08EF8FCD101E000F00CF8BDE8F183E7
:1028C00000240046FFF4FF11003801400024F4000A
:1028D000E00C0246816941F0080181617047296876
:1028E00051E8001F2A6821F4807142E80010002896
:1028F000704700002DE9F84300F0A2F846D1A08906
:10290000002835D0B80633D500F046F80880A86D09
:10291000821C00F06FF812D0F90748BF5FEAC85276
:1029200000F040F803D5F10701D500F05BF800F0A6
:1029300042F820B1284600F0CCFA0020606360889D
:102940000028DFD1FFF7CBFFFCD100F069F8FCD104
:1029500000F094F809D100F081F844BF1021016221
:102960002188284600F0B6FA02E0284600F00AFA6C
:10297000608868B1A18988420ADA00F044F8FCD185
:102980004D48A06100F024F8FCD101E0FFF7A2FF60
:10299000BDE8F183004400402968486AA96D09EA4E
:1029A0000000704705D501210162606B40F0010015
:1029B0006063B8077047780708D5F10706D52A681D
:1029C00004201062606B40F002006063606B70472F
:1029D000296851E8001F2A6841F0200142E80010F0
:1029E000002870472A6802201062606B40F00400E3
:1029F00060637047AA656088411E61802868C76966
:102A000017F0070F7047286800F1080252E8001F0E
:102A100000F1080921F0805149E8001000287047B2
:102A2000286800F1080151E8001F00F10803204860
:102A3000014043E8001000287047000000FD0F002F
:102A40000546286805F15C04B4F80490C76901469E
:102A5000D1F800808668216B22297047002121610E
:102A6000286850E8001F024621F0100142E80010DB
:102A70000028F5D12868C169CA0670472020206364
:102A80000021A1610020606128680C4988420CD0B7
:102A90004068010209D5286850E8001F024621F06D
:102AA000806142E800100028F5D1206901287047B4
:102AB000FEFFFFEFD526000825270008002400466A
:102AC00010B5DFF81C43DFF81C0300F04EF822625B
:102AD0006262A26262662046FFF7AAF808B100F0BF
:102AE00009FE0021204600F02DFE08B100F002FE94
:102AF0000021204600F031FE08B100F0FBFD204629
:102B000000F002FE18B1BDE8104000F0F3BD10BDAA
:102B100010B5DFF8D442DFF8D40200F026F8E26105
:102B200022626262A2622046FFF782F808B100F0DA
:102B3000E1FD0021204600F005FE08B100F0DAFDBD
:102B40000021204600F009FE08B100F0D3FD204628
:102B500000F0DAFD08B100F0CDFDA54901F2DC502E
:102B600000220260204601221CE120600C204FF46C
:102B7000E131002260616160A260E2602261A261D5
:102B8000704770B596B004461421684600F038FED0
:102B9000402106A800F034FE20689249954C964DDD
:102BA000964E884223D14FF40072002106920F9175
:102BB00006A800F029FE08B100F09CFDF06940F085
:102BC0004000F061F06900F0400000F05AF84FF466
:102BD000006100F04DF8082100F043F800224FF4A6
:102BE000806000F033F8082200F036F82CE07F49CE
:102BF000884229D1012200210692079106A800F0FF
:102C000003FE08B100F076FDB06940F48040B06189
:102C1000B06900F4804000F034F84FF4805100F0C7
:102C200027F8072100F01DF800224FF4807000F013
:102C30000DF8072200F010F8002200212E2000F0ED
:102C4000F4FE2E2000F018FF16B070BD0221029293
:102C5000039200900191704704926946204600F06B
:102C60006BBF0222049101926946284600F064BFBE
:102C700002F0010205920598009100210291039152
:102C8000704705900598316841F002013160326863
:102C900002F0020205920598316841F001013160AD
:102CA0003268704738B501684E4B554A514C52480E
:102CB00099420ED155684FF4006125F040055560EA
:102CC00000F0F1FF20464FF48061BDE8344000F091
:102CD000EABF464B994211D1116821F4804111603D
:102CE0004FF4805100F0DFFF4FF48071204600F078
:102CF000DAFF2E20BDE8324000F0C9BE31BD38B544
:102D00000446394D2846FEF7D7FF6C602846FEF78B
:102D10008FFF10B14FF0FF3032BD3A480021016003
:102D2000002032BD10B5324C40F2DC51204600F09C
:102D300067FD04F2DC500022026010BD0A46014625
:102D400080B54FF0FF332848FEF7DBFF08B14FF0A6
:102D5000FF3002BD264910B501F2DC5253881488B9
:102D6000A3420CD0C95C0170508840F2DC51401C79
:102D700083B28B42A8BF00205080002010BD4FF0CE
:102D8000FF3010BD10B51A49B1F8DC3540F2DC5403
:102D90005B1C9AB2A242A8BF0023A1F8DC359BB20B
:102DA00001221944BDE81040FEF7FBBFF8B50C4600
:102DB0001546012818BF022802D04FF0FF30F2BD9F
:102DC0000026074F07E04FF0FF330122A1193846D4
:102DD000FEF797FF761CAE42F5D32846F2BD000001
:102DE000E00A002000240046740B00200038014057
:102DF000D800002000000242000402428C0C02466F
:102E0000A40C0246B406002001484068704700BF89
:102E10000000002070B50446FFF7F6FF06462CB30D
:102E200004F14C05287A022802D02021E9601BE039
:102E30002068416941F00401416105202872206841
:102E400001698A0414D4FFF7DFFF801B0628F6D33C
:102E5000E868032140F01000E86029722879010633
:102E600002D5A96A0120087300202870012070BDD6
:102E7000416941F0020141610420287222684FF447
:102E8000FE410120D16000F018F80020287070BDCC
:102E900030B100F154010A78022A03D020204860A2
:102EA0000120704704220A700068416941F4005112
:102EB00041F0040141610020704728722979080619
:102EC00005D5A86A01210173226800219164704729
:102ED0000000704770477047704770472DE9F84F02
:102EE000040044D0DFF80477D7F81C90D7F828A066
:102EF000207809F00C090AF00305C1072AD5B9F1B9
:102F0000080F04D0B9F10C0F08BF032D62D160681F
:102F100000282CD0B9F1080F1CD13968A068012213
:102F200021F48811014341F4803139603868DFF8B9
:102F3000DC16DFF8D436000D00F001008240B1FB52
:102F4000F2F1DFF8C0261160186800F01FFF0028BA
:102F500040F0E9812078810712D5B9F1000F04D043
:102F6000B9F10C0F08BF022D57D12069002800F0DD
:102F7000DA813869616920F4F81040EA014038616B
:102F80002078DFF88C86DFF88C56010740F1C0808E
:102F900028684FF0000A41070AD428684FF0010A58
:102FA00040F004002860296801F0040100910098B5
:102FB000D8F80010C80751D400F0DDF90646D8F85B
:102FC0000000C1074AD4FFF71FFF801B0328F6D378
:102FD00003207FE1606888B13A68A16822F4881212
:102FE0001043084300F0C4F9064638688103B1D4A1
:102FF000FFF70AFF801B6528F7D3E9E7386820F45C
:10300000881000F0B5F9064638688103A2D5FFF7AD
:10301000FBFE801B6528F7D3DAE7206978B13968B1
:1030200041F480713960FFF7EFFE054638684105CD
:103030009FD4FFF7E9FE401B0328F7D3C8E73868A1
:1030400020F4807000F094F905463868410597D562
:10305000FFF7DAFE401B0328F7D3B9E7EE6DA0694E
:10306000002843D040011AD5E16906F08050814222
:1030700011D031010FD526F08066EE65FFF7C4FE52
:103080008346E86D010106D5FFF7BEFEA0EB0B00FD
:103090001528F6D39CE726F08050E6690643A06920
:1030A0000643EE65FFF7B0FE0090B346A669E86DF3
:1030B00010EA460F06D1FFF7A7FE0099401A15281F
:1030C000F4D385E786F010562BEA060BC5F85CB002
:1030D000FFF79AFE8346E86D10EA460F16D0FFF719
:1030E00093FEA0EB0B001528F5D371E726F01056E0
:1030F000EE65FFF789FE0646E86D10F0904F05D0AB
:10310000FFF782FE801B1528F6D361E700F028F94F
:10311000217848076CD529684FF0000A48070AD47F
:1031200029684FF0010A41F004012960286800F085
:10313000040000900098D8F80010C8070CD400F0E4
:103140001AF90646D8F80000C10705D4FFF75CFE5F
:10315000801B0328F6D33BE7E06841F2893828B3A7
:10316000E96D21F080010843E865FFF74DFE064652
:10317000E86D810705D4FFF747FE801B4045F7D374
:1031800026E7207B010608D5E86D01052ED4FFF760
:103190003BFE801B4045F7D31AE7E86D010525D5B6
:1031A000FFF732FE801B4045F7D311E7E86D20F0B2
:1031B0008100E865E86D20F00400E865FFF724FE73
:1031C0000646E86D810705D5FFF71EFE801B4045CA
:1031D000F7D3FDE6E86D010608D5E86D010505D5D4
:1031E000FFF712FE801B4045F7D3F1E600F0B8F878
:1031F000206A00286DD0B9F10C0F6DD00228386814
:1032000020F08070386053D1FFF7FEFD0546D7F8F7
:1032100000A0FFF7F9FD401B0328E6D25FEA8A1001
:10322000F5D4626A032A07D14FEA1A51DFF8DC03AA
:1032300001F00101C84001E0DFF8C403A36ADFF830
:10324000D813B0FBF3F088422CBF0C210021D7F833
:103250002890DFF8C8035B1E00EA0900024311430F
:1032600041EA032141F48021B962E06A216B401EEA
:10327000491E40EA4120616B491E40EA0140A16BB2
:10328000491E40EA01607863E06B10B100F062F81B
:10329000B862386840F0807000F06AF80446386818
:1032A000810116D4FFF7B0FD001B0328F7D38FE68A
:1032B000FFF7AAFD04463868810105D5FFF7A4FD94
:1032C000001B0328F7D383E6B86ADFF854130840DD
:1032D000B8620020BDE8F28F012824D0B86A796B6B
:1032E000636A00F003029A4201BFC0F30220401C4F
:1032F000A26A904217D1E26AC1F30800401C9042D2
:1033000001BFC1F34620401C226B90420BD1626B7F
:10331000C1F30640401C904201BFC1F30660401C4F
:10332000A16B884201D00120D4E7B86BE16BC0F3F8
:10333000CC008142CDD0B86A20F01000B862FFF70F
:1033400063FD0546FFF760FD401BFBD0E06B00F01E
:1033500001F8BDE7C000B863B86A40F010007047DC
:10336000BAF1000F03D0286820F0040028607047ED
:103370003860FFF749BDD8F8001041F00101C8F8E6
:103380000010FFF741BD2DE9F0410400884637D019
:10339000DFF89052286800F00F00404509D22968F4
:1033A000090948EA01112960286800F00F0040452A
:1033B00026D12178880609D5DFF840221368A16953
:1033C000E06923F017030B43034313602178DFF810
:1033D0001C72C80742D53868616803290CD1800186
:1033E0006BD5F96901F00C010C290CD0B96A0120E8
:1033F00060F31551B96206E0022902D1800302D4BC
:103400005BE0410559D5FA696068920840EA82029A
:10341000FA61FFF7F9FC06466068F96901F00C01F2
:10342000B1EB800F08D0FFF7EFFC801B41F2893130
:103430008842F1D3032052E003280FD1B86A20F468
:103440008010B862FFF7E0FC0646B86A410205D476
:10345000FFF7DAFC801B0B28F7D3EBE7396A226809
:103460000020930704D5C908C800A16801430120C2
:10347000530704D521F07000E168014301201207D1
:1034800005D5206921F4E06141EA001100E000B1B6
:1034900039622078C10644BF60697862296801F00A
:1034A0000F0188450BD22868000948EA00102860FF
:1034B000296801F00F01414501D001200FE000F023
:1034C00010F83A6A58494F4B02F00702895CC8402D
:1034D00018604D480068BDE8F04100F057BCBDE8F9
:1034E000F0814249C86910F00C0001D1444870478E
:1034F000082818BF00F036B809684448090D01F0E3
:103500000101C840704780B5FFF7EBFF47490968E4
:10351000454A3C4B01F00701515CC840186002BDB0
:1035200080B5FFF7F0FF414A0CE080B5FFF7EBFFF5
:103530003E4A13683E49C3F3022207E080B5FFF715
:10354000E2FF3C4A13683A49C3F30212895CC8405F
:1035500002BD10EE100A491CB0FBF1F010BD364858
:10356000046807E010B5FFF7FAFFBCEEC00AC4F329
:103570000661EEE71D48416BC1F30801491C00EEEE
:10358000101A816AB8EE400AC1F30222521C00EE02
:10359000902AF8EE600ACA0643BF826BC2F3CC02DF
:1035A00001EE102A9FED121A01F00301B8EE411A44
:1035B000022902D0032903D00DE0DFED0E1A0CE042
:1035C00000681249000D00F00100C14001EE901AA0
:1035D000F8EE611A01E0DFED061AC1EEA00ADFED98
:1035E000061A01EE210A20EE800A7047000C0246FE
:1035F000000000000024744B00000039000E024659
:103600000024F4000C000020080000200048E8011D
:1036100028080246940C024601127A00E0F8FFFFE7
:10362000FCFFF8FF00200240B0470008200C0246D3
:103630009C800008240C0246340C024680B500F041
:10364000EFFB00F013F800F005FCFFF739FAFFF785
:103650005FFA00F0A1FC00F0FDFC00F00BFD00F0B3
:103660006EFC00BF24A000F0C9FFFEE780B598B053
:10367000402108A800F0C4F82021684600F0C0F8F6
:103680004FF4803000F0CEFF08B100F033F8002294
:103690000A920F924FF480310322099111924FF058
:1036A0008061082209200E911392089002210022C5
:1036B00010911291149115911691179208A8FFF785
:1036C0000DFC08B100F016F83F2100910021032203
:1036D0000291049101920421002206910392059225
:1036E000079201216846FFF74EFE08B100F002F88C
:1036F00019B000BD72B6FEE74C54452054455354F2
:1037000020444F4E450D0A0010B500F184010A789F
:10371000012A01D1022010BD01220A7024234B602E
:10372000026813681468640864001460002242662A
:10373000006823F00053202203604A6000230B70CE
:10374000002010BD70B500F01FF801D1022070BD3F
:1037500000F020F822F0604209E070B500F014F8A3
:1037600001D1022070BD00F015F822F06062114313
:103770008160204600F01CF82068202100220660AD
:1037800069602A70002070BD044604F18405287821
:10379000012870470120287024226A60206806688A
:1037A0000268520852000260206882687047000078
:1037B00030B5416E11B90121012214E0016800BF4A
:1037C0000FF22C040CA38A688968520E02F00702DB
:1037D000490F655CA45C595C9A5CED00E40095FBC4
:1037E000F1F194FBF2F268304180028030BD0000BC
:1037F000010101030701000008040204080101019E
:10380000002200F03DBF00002DE9FC47064630785D
:10381000DFF8EC71C10705D53A687068920840EA94
:1038200082023A603178880705D53968B06821F09E
:103830000C01014339603178480705D53968F068D3
:1038400021F44061014339603178080705D53968B2
:10385000306921F44021014339603178C80605D52B
:103860003968706921F44011014339603178880664
:1038700005D53968B06921F44001014339603178D8
:10388000480605D53968F06921F0004101433960E7
:103890003168DFF87041C8050DD57968306A21F4C8
:1038A000405101437960316AB1F5405F03D120682E
:1038B00040F4003020603168880505D5B968706A29
:1038C000890840EA8101B9603168480505D5B968C1
:1038D000B06A21F018010143B9603168080505D5C7
:1038E000B968F06A21F0C0010143B9603168C804C9
:1038F00005D5B968306B21F440610143B960316886
:1039000088040DD5B968706B21F4E0410143B960BA
:10391000716BB1F5005F03D1206840F48030206006
:103920003168480458D5D7F81090B06B4FF00008B4
:1039300009F4407981454FD0E16E48070AD4E16E21
:103940004FF0010841F00401E166E06E00F0040070
:1039500000900098DFF8B050286840F0010028601F
:10396000FFF752FA82462868C10707D4FFF74CFADE
:10397000A0EB0A000228F6D903203FE03869B9F12C
:10398000000F20F4407009D0B9693A6942F48032DE
:103990003A613A6922F480323A61B961B16B01430C
:1039A0003961DFF8681011EA00090ED0FFF72CFA30
:1039B0000546386910EA490F07D1FFF725FA401B81
:1039C00041F289318842F4D3D6E7B8F1000F03D031
:1039D000E06E20F00400E066306801040DD53A691D
:1039E000F06B22F4402202433A613969F06B01F432
:1039F0004021814218BF012000D10020BDE8F68798
:103A0000E00C0246280C0246280802460100002469
:103A1000414B19684FF6FF020002114000F4E060CC
:103A200008433E4908431860704770B53A4B1C681C
:103A3000C4F302230124C3F10705052D2EBF0F2572
:103A400004FA05F56D1E1E1D072E34BF0023DB1E74
:103A50002940994004FA03F35B1E1A4011430901FF
:103A6000020002D42E48815470BD2E4B02F00F028A
:103A70001A4402F8041C70BD010007D4012200F0B2
:103A80001F018A40284B400943F82020704701005D
:103A90000BD4012200F01F018A40244B400943F857
:103AA0002020BFF34F8FBFF36F8F7047401EB0F1E0
:103AB000807F07D21E49486000228A600B6843F06D
:103AC00003030B60B0F1807F8041C043C00F70479B
:103AD0001849174A04281ED8DFE800F00811141D01
:103AE0000300106840F0040010607047136823F072
:103AF00004031360086820F44000086070471368EE
:103B0000012001E01368022023F0040313600A6817
:103B100060F397520A6070470CED00E00000FA0570
:103B200000E400E018ED00E000E100E080E100E0EA
:103B300010E000E0E00C02462DE9F04F4FF0000CE1
:103B40008E4A8F4BDFF83C824FF00F0906460F4636
:103B5000A2E0012404FA0CF414EA010058D04FEA60
:103B60004C0103258D406FEA050E7D6805F0030AC0
:103B7000BAF1010F1CBF05F00305022D13D1B56882
:103B8000D7F80CA00EEA05050AFA01FA4AEA05057B
:103B9000B560756825EA04047D68C5F3001505FA6B
:103BA0000CF52C4374603D79BC6805F00305032DCA
:103BB00008BF012C05D0F5688C400EEA05052C43A2
:103BC000F4603C7904F00304022C14D14FEADC04C5
:103BD00006EB8404D4F820A04FEA8C0505F01C0500
:103BE00009FA05FB2AEA0B0AD7F810B00BFA05F51B
:103BF00045EA0A05256234680EEA04053C7904F0BA
:103C0000030404FA01F129433160796811F4403F5B
:103C100040D04FEA9C01DFF870A158F821E04FEA4C
:103C2000CC040AEA962A04F0180409FA04F52EEAEC
:103C300005050AFA04F444EA050E48F821E0D3F831
:103C400000E07C68C14301EA0E0EE50248BF40EA8D
:103C50000E0EC3F800E0D3F804E07C6801EA0E0E13
:103C6000A50248BF40EA0E0EC3F804E0D2F804E013
:103C70007C6801EA0E0EA50348BF40EA0E0EC2F8AA
:103C800004E0D2F800E07C6801EA0E01E40348BFDA
:103C9000014311600CF1010C396831FA0CF07FF42A
:103CA00058AFBDE8F08F2DE9F04F02460027344BA6
:103CB000DFF8C8804FF00F09DFF8C8A053E00120FB
:103CC00000FA07FC1CEA01004CD04FEA970EDFF81F
:103CD000B8B05AF82E60FD000BEA922B05F01805DB
:103CE00009FA05F426400BFA05F5AE4216D1D8F8CC
:103CF0000050C0430540C8F80050D8F804600640A2
:103D0000C8F804605D6805405D601E68304018605A
:103D10005AF82E0020EA04044AF82E4003207C00C2
:103D2000A0401468FD0802EB850E04431460DEF821
:103D30002040BD0005F01C0509FA05F5AC43CEF89E
:103D40002040D2F808E0C04300EA0E0EC2F808E0B6
:103D5000546824EA0C0CC2F804C0D2F80CC000EA83
:103D60000C00D0607F1C31FA07F0A8D1BDE8F08FBD
:103D70000AB181617047816270470000802002466D
:103D800000200246602002467F7F2F00F8B50446DF
:103D90001F4D2878002100282ED01E4A12681E4B85
:103DA0001E68770702D54FF47A710DE01B4B1B6834
:103DB00013F4400306D0B3F5800F08D0B3F5000F1D
:103DC0000ED015E04FF4FA51B1FBF0F00EE04FF4D5
:103DD0007A72B2FBF0F24FF4FA43B3FBF2F107E070
:103DE0004FF47A71B1FBF0F04FF40042B2FBF0F106
:103DF0000846FFF75BFE08B10120F2BD0022214614
:103E00004FF0FF30FFF711FEAC600020F2BD00BFA5
:103E1000000000200C00002010E000E0E00C024652
:103E200080B50B48016841F4807101600320FFF701
:103E3000EFFD00F049FC0420FFF74AFE0F20FFF7DA
:103E4000A5FF08B1012002BD00F0B6FC002002BDB4
:103E50000020024038B586B0142101A8FFF7D0FC3D
:103E60004648016848F29105454C41F00201016065
:103E7000026802F0020200920099026842F0010218
:103E80000260036803F00103009300990268294669
:103E900042F0040202600068002200F0040000907A
:103EA000009800F049F80121029100220195039247
:103EB000049201A92046FFF73FFE07B030BD012262
:103EC00000E0002280212E48FFF752BF10B52C4C95
:103ED0000122102100F030F82A4800F08FFB00F09A
:103EE00055F800F027F8642000F086FC012200F06D
:103EF00022F8012200F04BF8C82000F07DFC00F011
:103F000019F84FF4AF7000F077FC00F03FF8642030
:103F100000F072FC0C24FFF7D2FF4FF4FA7000F0AF
:103F20006BFCFFF7CEFF4FF4FA7000F065FC641EE7
:103F3000F1D110BD002201212046FFF719BF10B5B5
:103F4000114800F05BFB0E4C00F020F8642000F0FC
:103F500053FC012200F01BF84FF42F7000F04CFCD2
:103F600000F014F8FFF7ABFF1E244FF47A7000F056
:103F700043FC641EF9D1BDE81040A2E78C0C024658
:103F800000040242287F00084C7F000800224FF402
:103F900000412046FFF7ECBE18B587B01C22002177
:103FA000684600F03DFC284C28482060FF20E06077
:103FB0004FF0804000217F22E0616160A2602161BA
:103FC0006161A16121626162204600F033FC08B1A9
:103FD000FFF790FB00210091039104910591694640
:103FE000204600F028FD08B1FFF784FB00220021E5
:103FF000204600F0DDFC08B1FFF77CFB08B010BDE7
:1040000010B590B0044640220021684600F008FC3C
:1040100021680E4A914215D14FF480434FF400714C
:1040200000930E916846FFF7EFFB08B1FFF762FBC4
:104030000748016841F400110160006800F40010B5
:104040000090009810B010BD580C00200078004679
:10405000A80C024680B5002000F00CFD08B1FFF767
:1040600049FB00F013FD18B1BDE80140FFF742BB6A
:1040700001BD00002DE9F04FA3B000200090DFF853
:10408000005402260027FFF721FF05F51C7ADFF810
:10409000F4B30FF238480FF22049322000F0ACFBA5
:1040A000782000F0F2F804460A22294609A800F018
:1040B000FDFC0146484600F0A1FA00F0E2F809A82C
:1040C00000F0CEF909A9404600F098FA00F0D9F8BE
:1040D00009A800F0C1F909A90FF2044000F08EFA16
:1040E00000F0CFF809A800F0C6F909A90FF20440C2
:1040F00000F084FA00F0C5F809A800F0B8F909A9A1
:104100000FF2FC3000F07AFA652109A87F1CFFF756
:1041100077FBFF2C3DD00A2C42D0002C1DD15846F5
:1041200000F06CFA00F0ADF8684600F055F9009820
:10413000632808D041000246713949B20BF12C00C6
:1041400000F05CFA03E00BF15C0000F057FA9FA06E
:1041500000F054FA0BF580702CE0FBD0012C0CD051
:10416000022C10D0032C11D0042C18BF052C04D025
:104170000A2C15D0FF2C0CD015E000F029F90026F0
:104180000BF1840016E00BF1B00013E00BF1D80046
:1041900010E00BF5947000F031FA0BF5B07009E007
:1041A0000FF2683006E021460FF2803000F026FA68
:1041B0000BF5CE7000F022FA0FF2903000F01EFAEC
:1041C000B521504600F013F9002830D151460FF2C6
:1041D000903000F013FA0FF2903100F04FF820B950
:1041E0000FF28C3100F04AF810B10FF28C3118E068
:1041F0000FF2903100F042F820B90FF2903100F048
:104200003DF810B10FF28C310BE00FF2A03100F04D
:1042100035F820B90FF29C3100F030F828B10FF2D8
:104220009C3101A800F052FC05E0012603E00BF5EB
:10423000F87000F0E3F901A800F0E5F8B8B900F073
:10424000F1F80121284601F07BF801280BD100F09C
:10425000F6F841F2883000F0CFFA08E04FF0FF3076
:1042600023B0BDE8F08F0FF2683000F0C7F9304698
:10427000002EF5D0032FFFF610AFEFE7504601F008
:1042800008BA652109A8FFF7BBBA2DE9F04F85B040
:10429000002603968DF81060DFF8E4B18246FEF741
:1042A000B3FD0546DFF8E011584600F0B2FFDFF835
:1042B000DC01DFF8DC11DFF8DC21029001910092D3
:1042C000DFF8D431DFF8D421DFF8D4115846FF27C6
:1042D0004FF47A7400F0EFFC04FB0AF4022870D16A
:1042E000584600F007FD022865D1FEF78DFD401B02
:1042F00058A7DFF8B0814FF6FF790EE0384600F09E
:104300007DF905E0002EF9D1404600F077F901264D
:1043100000F05EF8FEF778FD401BA04201D3CA45CD
:1043200011D103A9584600F04DFE0228F2D103989E
:104330006328E7D04100713949B20FF2A42000F0A0
:104340005DF900F045F80FF230220121584600F0E7
:1043500069FFFEF759FD401B9DF9107004E000F065
:1043600037F8FEF751FD401BA04201D3CA4517D1D3
:10437000584600F09EFE0128F3D1584600F07DFE1D
:104380000128EED1584600F034FE022808D07F1CE8
:1043900078B20128E3D1584600F04EFE0228DED064
:1043A000584600F086FE0746012818BF052808D1A8
:1043B000FEF72AFD05E0082802BF9BF8D270032F04
:1043C0001327384605B0BDE8F08F00000D0A000045
:1043D0004FF47A7000F010BA014610B500F02CF8D6
:1043E00000F0F0FD022808BF0024204610BDCAB22C
:1043F000014610B500F020F800F086FE022808BF44
:104400000024204610BD024610B500F007F800F069
:1044100040FF022808BF0024204610BD0121184893
:104420000224704710B500F007F800F0D2FF022810
:1044300008BF0024204610BD11480224704710B563
:10444000FFF7FAFF01F001F8022808BF0024204618
:1044500010BD00002E00000080B56422124902E069
:1044600080B51022114900F021FB002002BD80B56B
:1044700014220F49F7E780B510220E49F3E7000038
:10448000B8060020C87A0008092E0008252D00086B
:10449000552D00083D2D0008FF2C0008B91C000810
:1044A000112B0008847E0008F4060020C2060020BC
:1044B000C0070020580700204D6F64756C65204EC2
:1044C000616D653A2025730D0A00000050726F641B
:1044D0007563742049443A2025730D0A00000000DA
:1044E00046572056657273696F6E3A2025730D0A20
:1044F00000000000494D45493A2025730D0A00008F
:1045000049434349443A2025730D0A000D0A203ED1
:104510003E3E2053494D206973206E6F7420494EF2
:104520005345525445440D0A0D0A00000D0A203E21
:104530003E3E204D6F64756C652053494D20457299
:10454000726F723A2025640D0A00000043656C6C9E
:10455000756C6172204F70657261746F723A2000E1
:1045600025730D0A00000000534D41525400000015
:104570003531353033000000696E7465726E6574D4
:1045800000000000474C4F424500000035313530F7
:1045900032000000696E7465726E65742E676C6F10
:1045A00062652E636F6D2E70680000004449544FA1
:1045B000000000003531353636000000696E746544
:1045C000726E65742E6469746F2E7068000000004E
:1045D00050696E672057696C6C204E6F740D0A002D
:1045E0000D0A5369676E616C204C6576656C3A20E4
:1045F00025642064426D0D0A000000000EB4C0B5B1
:10460000024603A800210190009101AB012104485A
:1046100078440C30FBF7A5FD06BC5DF810FB00BF2D
:10462000553A000010B5134A116B01F480318142F4
:104630001BD01168104B21F48031084310601C68B6
:1046400032200E494443B4FBF1F1491C084601E015
:1046500068B1401E13681C04FAD540B101E031B1C5
:10466000491E106B0304FAD509B1002010BD0320C8
:1046700010BD00000C0802460C00002040420F0054
:1046800000B500BF130096469446103928BFA0E835
:104690000C50FAD85FEA417C28BF0CC048BF40F8F4
:1046A000042BC90728BF20F8022B48BF00F8012BB4
:1046B00000BD000037480168374A41F470010160CD
:1046C000364810607047000030B53549CB69354831
:1046D000354A03F00C03082B02D00C2B07D04BE01B
:1046E00010460A68120D02F00102D04044E08B6AC5
:1046F0004C6BC3F302256D1C00EE105AC4F3080581
:10470000C4F30664641C6D1C01EE104A00EE905A5E
:10471000DC0607D58C6BC4F3CC0401EE904AFBEEAB
:10472000E91A01E0DFED1A1A03F00303022B02D0AD
:10473000032B03D00AE002EE100A09E00868000D1E
:1047400000F00100C24002EE102A01E09FED102AA5
:10475000B8EE422AB8EE400AF8EE600A82EE000A8D
:1047600070EEA10A20EE200AF8EE410A80EE200A3F
:10477000BCEEC00A10EE100A0C4A1060096A00BFB5
:104780000BA301F00701595CC840106030BD000068
:104790000000000088ED00E008ED00E000000008E7
:1047A000000C02460024F4000048E8010C00002040
:1047B000000000000102030480B50E48816841F04A
:1047C00004018160816801F0040100910099026890
:1047D000002142F4801202600068002200F4801080
:1047E000009000984420FFF720F94420BDE80240E3
:1047F000FFF742B98C0C024638B50446FEF704FBBD
:10480000054614F1010F02D0044908780419FEF797
:10481000FBFA401BA042FAD331BD00BF00000020CC
:1048200010B5044610460A460146204600F048FFEF
:10483000204610BD70B504460120002C49D004F17B
:104840002C05697821B9002028702046FFF7D8FB95
:1048500002216970DFF850613068C10636D4CA2081
:10486000B0615321B161204600F052F8010028D117
:10487000F168DFF838010140F160F2686068216991
:104880000243A0690A430243F260E168A06841EA7A
:10489000004171603268616AA06A22F4F8520A43EA
:1048A00002433260204600F057F8010009D1F36856
:1048B000226AE16923F06043134362690B431343A7
:1048C000F360FF21B161020003D100E0002001216B
:1048D000697070BD84F82D0070BD70B50446324D0E
:1048E000286820F020002860FEF78EFA0646286827
:1048F00081060BD4FEF788FA801B40F2E93188422A
:10490000F5D32868810601D40320E3E7002070BDB9
:10491000F8B50546244C2068002641061AD42068C4
:1049200040F080002060FEF76FFA074603E00320A6
:10493000032685F82D00216848060BD4032E09D0E4
:10494000FEF762FAC01B40F2E9318842F3D32068D7
:104950004106ECD53046F2BD70B50446124D2868CC
:10496000002620F080002860E968880608D42046E8
:10497000FFF7B3FFA0B1032084F82D0003260FE05A
:10498000E86820F02000E8602046FFF7A6FF18B195
:10499000032084F82D000326E86840F02000E8603A
:1049A000304670BD000000000C780046BFFF8FFB52
:1049B0002DE9F04100F12C0630780C46154601280F
:1049C00008BF02202FD00120307002217170DFF863
:1049D0009870F86820F48060F8603968480614D44C
:1049E000FEF712FA8046386841070ED4FEF70CFA3B
:1049F000A0EB080000F01BF8F5D33868410704D499
:104A000003207070002131700DE0F8680121C008AA
:104A100045EAC005FD60BC60F86840F48060F8605D
:104A2000717000203070BDE8F081A0EB090040F209
:104A3000E9318842704710B50A6848680C4B024358
:104A40001A608C68CA688869084B144304435C6028
:104A50001A680869496922F0FF12024342EA0142DA
:104A600000201A6010BD00000C780046207C004633
:104A70001C78004610B500F010F801D5012010BDDB
:104A8000136823F004031943116010BD0648016840
:104A900041F00101016000207047034A136801469C
:104AA0000020DC07704700000004034001B55AB144
:104AB00011F8013B521E00F8013B03B1F8D111007F
:104AC0001CBF002200F0FCFD01BD00000CB430B59D
:104AD00083B00A4606A90291044600250194009578
:104AE00002AB01A9084878441E30FBF73AFB019A53
:104AF000157000284EBF04460198041B204603B0E1
:104B000030BC5DF80CFB00BFF7C8FFFF70B5024674
:104B100015780023002400202D2D0AD10123521CDA
:104B2000012406E012F8016B0A25641C05FB0060F5
:104B300030381578303D0A2DF4D301B10C7003B133
:104B4000404270BD002381423CBF4FF0FF331B1A2F
:104B5000591A4018101870472DE9F24F82460AF58D
:104B6000B2709AB0416893461C46249F88470190D2
:104B70000BF10F024FF47A5042434FF4E13100261B
:104B800092FBF1F0B84238BF384624900025DFF898
:104B90001C790DF138090DF1080868206843391DAA
:104BA00029F815600844FCF7B7FA28F815006D1CC1
:104BB000182DF2DB5FEA0B0008BF002C51D04FF438
:104BC00080710AF5B670FEF71BFE0AF5B27A02E0B4
:104BD000521C182A1ADBDAF8040080470146249A8E
:104BE0000198FFF7AFFF002836DDDAF800106846BD
:104BF00088470028EFD19DF800001A998855761C47
:104C000036B25FEA0B0224D10022682101FB02F0D8
:104C100039F812E09DF800C03B189E449EF80450FD
:104C2000AC451CBF002529F8125039F812509DF8E8
:104C300000E02B441B799E45CAD16D1C29F8125007
:104C400038F81230ADB29D42C2D338580442BFD0BA
:104C50000BE05E45BFDB04E0BBF1000F03D0002E8C
:104C600001DD304601E04FF0FF301BB0BDE8F08FB2
:104C70002DE9FC4105460C0016461F466FF0010861
:104C800008BF4FF4AF7400F001FBD5F8602181B28A
:104C90003046904700280BD4C820FFF7ADFD0094A4
:104CA0003B46002205F5B6712846FFF755FF8046C2
:104CB0004046BDE8F681F0B570B10C000CD0140090
:104CC0000AD01C0008D0059C250005D0069D2E00AA
:104CD00002D0079E370001D14020F0BD00F5A8703A
:104CE00001604260836004614561C6600220F0BDDE
:104CF000000000002DE9FC4780460020202788F8AE
:104D00003B010025002200230A214143414401F5D3
:104D10009F71401C0A704B704D808A80CB800028A8
:104D2000F2DD08F5A874E06880472168884700280C
:104D300040F0F880A06940254FF0000A8047814686
:104D40007AA6A069804701464FF4FA724846FFF7F9
:104D5000F9FE002809D54223324600F02BF905461A
:104D6000A0690AF1010A804781464FFA8AF00A28B1
:104D700063DA022DE5D1404600F0F9F9064608F560
:104D8000A471404600F0FFF90546422369A200F0F5
:104D900011F981465FF0420368A24FF4AF714046BB
:104DA0002E43FFF765FF49EA060606435FF042031C
:104DB00064A200F0FFF8064308F5B6750FF28829E3
:104DC000022E42D15FF0420361A200F0F3F8022804
:104DD00006D100F0F3F801460A224046FFF766FECE
:104DE0005FF042035DA200F0E5F8022807D100F071
:104DF000E5F80146322208F10A00FFF757FE422388
:104E000059A200F0D7F8022807D100F0D7F80146E0
:104E1000642208F13C00FFF749FE422355A200F04E
:104E2000C9F80646022E10D100F0C8F80146322219
:104E300008F1A000FFF73AFE09E0022D9BD0DFF851
:104E40008806FFF7DBFB042758E0022E56D1A06945
:104E500080470646A1698847801BB0F5FA6FF9D3F1
:104E600048F242044FEA040345A241F27C5100F0AB
:104E7000A3F802282FD100BF44A1284600F009FC66
:104E800000283BD0FF2088F8D200234643A200F040
:104E900091F8022807D100F091F80146322208F17A
:104EA000D600FFF703FE42233FA200F083F802285A
:104EB0000FD100F083F83A21FCF7F4F818B110F89C
:104EC000011F2029FBD00146322208F58470FFF72C
:104ED000EDFD022712E0B0F5004F0FD100F0A3F86E
:104EE0000123002229464046FFF736FE01A908F2B9
:104EF0006D10FFF70BFE88F8D200082748F2420336
:104F00000FF2DC5244F2740100F056F8022818BF88
:104F100020274FF01E081E20FFF76EFCB8F1010895
:104F2000F9D100E010273846BDE8F68741540D0A54
:104F300000000000415456310D0A00004154453034
:104F40000D0A000041542B434D45453D310D0A00EB
:104F500041542B43474D490D0A00000041542B4357
:104F6000474D4D0D0A00000041542B43474D520D53
:104F70000A00000041542B4347534E0D0A00000025
:104F800041542B4350494E3F0D0A00002B435049DA
:104F90004E3A2052454144590000000041542B43F1
:104FA000494D490D0A00000041542B4943434944EF
:104FB0000D0A00004FF4AF71404659E649462846B5
:104FC00000F088BB7CB500F053F80FF220524FF48C
:104FD000AF71FFF74DFE0646022E08D10FF21851B1
:104FE00000F08EF86946801DFFF790FD286030467E
:104FF00076BD38B5044694F8D2004025FF2810D17C
:1050000048F242030FF2F842DFF8C01400F056FAFB
:10501000022805D000F007F8012300F008F800E0AE
:105020000225284632BD4FF47A7000907047002266
:1050300004F5B67120468FE51CB500F01AF80FF2A2
:10504000D042DFF88C1403E00D0A000044F2740132
:10505000FFF70EFE02280AD04FF47A700090012369
:10506000002204F5B6712046FFF776FD402016BDFC
:105070000D46044648F2420370473EB500F035F84D
:1050800015D148F242030FF2944200F078F802285A
:105090000DD10FF2944100F033F840B16B4601AAF4
:1050A0000FF28C4100F03CFB022808BF009DE8B2E3
:1050B0003EBD3EB500F019F815D148F242030FF29B
:1050C000804200F05CF802280DD10FF2804100F020
:1050D00017F840B16B4601AA0FF2784100F020FBAF
:1050E000022808BF009DE8B23EBD002104460191A0
:1050F000009194F8D200FF25FF2870470FF2644119
:1051000004F5B67000F0C5BA2DE9F0410D4616461B
:10511000DFF8BC7348F24208044643460FF2F0320F
:105120003946FFF7A5FD43460FF24042394600F0ED
:10513000C5F90746022F15D1FFF7E0FFC11D00F0AA
:1051400064F80FF24C584146FFF739FF022403E0A0
:10515000414600F0ADF9641E38B1002CF8D101468B
:1051600000F053F83846BDE8F0814027FAE74223C3
:105170000FF204424FF4AF717AE5422342464FF4F6
:10518000AF71204674E5F8B50C4642230FF2F032B9
:105190004FF4AF710546FFF76BFD05F5B6760228B3
:1051A0000AD10FF2E831304600F073FA0021801D79
:1051B000FFF7ACFCC5F8480142230FF2D8324FF498
:1051C000AF712846FFF754FD0546022D1BD10FF2A3
:1051D000D031304600F05DFA861D00213046FFF7E1
:1051E00095FC07460021B01CFFF790FCFFB2C0B24F
:1051F000022F04D1022814BF0120032002E002285C
:1052000018BF002060602846F2BD32462846FFF7EE
:105210004DBC08B10A0001D140207047C0F86811A8
:10522000022070472DE9FF4100F02DF8DFF8A4823D
:1052300000F11A0100962B460FF26C32404600F046
:1052400083FAFFF79AFF07460FF278320D214046A6
:1052500000F07AFAFFF791FF022F10D192A00021FF
:1052600003910290019000962B46DFF86C224FF4D8
:105270008071404600F068FAFFF77FFF0746384626
:1052800004B0BDE8F081044616460D463046FBF7F3
:1052900043BF2DE9F041FFF7F6FFDFF8387200F168
:1052A000190133460FF22C32384600F04DFA4223F2
:1052B0003A46FFF764FF0646022E2FD194F83B01D1
:1052C000022827DC2B460FF228321821384600F03E
:1052D0003BFADFF8F88100F0EEF800F022F8022E39
:1052E00018D10FF21C321821384600F02DFA00F0C8
:1052F000E2F800F016F8022E0CD100F01CF808B904
:10530000FF200CE0401C00F0E3FA00F00EF8401C17
:1053100084F83B014FF4FA70FFF76EFA3046BDE8AF
:10532000F08106460A20FFF767BA04F23B114855A0
:1053300094F83B0170472C2104F5B670FBF7B2BE20
:105340002DE9FE4305460E46DFF888410FF2B022F4
:105350000B21204600F0F8F942232246DFF86C11B9
:105360002846FFF785FC022830D156A7394605F5B7
:10537000B67000F0AFF904460FF298280FF28C29AE
:1053800003E0394600F094F80446FCB14946204653
:1053900000F07FF90028F4D00021019100916B46C4
:1053A00001AA4146204600F0BBF9022804BF01983B
:1053B000B042E6D10099AA190FF2682082F83B1199
:1053C0000099FFF71BF90098C0B200E0FF20BDE88C
:1053D000FE832DE9F04190B0044642230FF25C2297
:1053E000DFF8E8104025FFF743FC022829D104F537
:1053F000B6700FF258270FF268281CE02221FBF745
:1054000051FE060015D02221701CFBF74BFE040054
:105410000FD0841B641E3F2C88BF3F242246711C82
:105420006846FFF743FB0020694608553846FFF7FA
:10543000E5F805F10A00414600F02BF90500DDD141
:105440000225284610B0BDE8F0812DE9F843054655
:10545000DFF880400FF214221B21204600F074F97F
:10546000DFF878603346224641F27C512846FFF748
:10547000FFFB0746022F13D1062405F5B6780FF27D
:1054800008294FF4AF700090334600224146284669
:10549000FFF762FB41464846FFF7B0F8641EF0D1C3
:1054A0003846BDE8F283000000000000D871000813
:1054B000002000F00FB942233A4641462046FFF74C
:1054C000D7BB00000D0A0000907D0008606102005B
:1054D00090D60200E0090020047F000810000900B7
:1054E00041542B4346554E3D310D0A0041542B4348
:1054F00053510D0A000000002B4353513A000000A5
:1055000041542B43474154543D310D0A00000000E3
:1055100041542B434F50533D300D0A0041542B430F
:105520005245473F0D0A00002B435245473A0000C1
:105530002B435245473A2025642C25640000000087
:1055400041542B43475245473F0D0A002B434752D6
:1055500045473A002B43475245473A2025642C25BE
:10556000640000002B434F50533A000041542B433A
:105570004F50533F0D0A0000415426460D0A0000CB
:1055800041542B4950523F0D0A0000002B49505204
:105590003A00000041542B4946433F0D0A000000E9
:1055A0002B4946433A00000041542B434744434FA4
:1055B0004E543D25642C224950222C222573220D65
:1055C0000A00000041542B434744434F4E543F0DC3
:1055D0000A00000041542B434744434F4E543D3191
:1055E0002C224950222C20222573220D0A00000073
:1055F00041542B43474143543D312C25640D0A004F
:1056000041542B43474143543F0D0A002B4347412C
:1056100043543A002B43474143543A2025642C25F8
:105620006400000041637469766520537461746599
:10563000202D2D2D2025640D0A00000041542B4300
:105640004750414444523D310D0A00004950204129
:105650006464726573733A2025730D0A00000000BC
:105660002B434750414444523A20000041542B51AF
:1056700050494E473D312C22382E382E382E3822B4
:105680002C31302C350D0A0025730D0A0000000066
:105690002C0070B50D462C7834B970BD11F8013F5F
:1056A0001678B34206D0401C2146FBF7FBFC28B11C
:1056B00001462A4612F8013F002BEFD170BD0000D1
:1056C0004018491C1CBFB1F1010100F8012DF9D1AE
:1056D0007047000038B504000D460BD0294620461F
:1056E00000F0FDF80444207848B90C48002101601E
:1056F000002032BD09490C68002CEFD132BD29468B
:10570000204600F0FDF82118087810B1002201F8B9
:10571000012B02480160204632BD00BF880C0020EA
:105720000DB4C0B50A4604A800210190009101AB58
:1057300003A9044878440C3000F01CF906BC5DF85D
:1057400010FB00BF77B9FFFF08B438B585B009ACCE
:1057500000250494039500290EBF01950190491E70
:105760000291009504AB01A9074878441A30FAF772
:10577000F8FC019901B10D70002858BF039806B0DC
:1057800030BC5DF808FB00BF27BCFFFF2DE9F84FD8
:1057900084B00E4617460BB100221A600446A0469C
:1057A00001E008F1010898F8000000F079FF0028F6
:1057B000F7D198F800002D2816BF2B2818F8015BA8
:1057C0002B25002F019603D4012F01D0252F03DBB9
:1057D000002E56D0346054E0002F0CDD102F04BF93
:1057E00098F80000302802BF98F8010040F020002F
:1057F000782811D10CE098F80000302818BF0A274B
:105800000AD198F8010040F02000782803D1102731
:1058100008F1020800E00827CDF80C8001E008F14B
:10582000010898F800003028F9D0064E7E4414365E
:105830004FF0000906F12800CDF80880CA468DF81F
:1058400000000CE0AC24000001469DF80000081A9E
:10585000CA465FFA80FB07FB09B908F1010898F80E
:10586000000000F027FF01463A4606F12800FBF74A
:105870005DFC0028E8D10399414504D1019800B1AD
:105880000460002020E00299F05DA8EB0101091AF4
:10589000002910D406DCB9EB0B0103D3B1FBF7F000
:1058A000504508D0AFF30080049808B10121016091
:1058B0004FF0FF3903E02D2D08BFC9F10009019811
:1058C00008B1C0F80080484605B0BDE8F08F04E09C
:1058D00000E000000A220021F9E7002356E770B437
:1058E000044600E0641C23783BB10D462A7822B1BF
:1058F00015F8016BB342F9D1F4E7201A70BC704778
:1059000070B4044600E0641C23783BB10D462A784D
:10591000002AF8D015F8016BB342F8D1201A70BCF8
:1059200070470000034608460122C168491CC16057
:1059300000210068184703460846C1680269491CEF
:10594000521E002A0261C16003D4006801220021B6
:1059500018474FF0FF307047034608461146C268AB
:10596000521E11F1010FC26002D0006800221847D8
:10597000704700002DE9F84F9AB04FF0FF340091C6
:1059800000261B68019302920DF13F02249B8DF8C3
:105990001F30A04603961992814613E00398401CDD
:1059A0000390012200980021C847064600F078FEC7
:1059B0000028F3D1324669464846FFF7CDFF0298EA
:1059C000411C02910298007800F06AFE0028E5D19F
:1059D000029E307820B9404500DA404600F034BDE0
:1059E00025280AD1701C029001782A2903BF401C87
:1059F000029010F8011D002110E00398401C039054
:105A0000012200980021C84731788842D7D0024649
:105A100069464846FFF7A0FF0020DCE78DF81C1020
:105A200000210591DFF8143A0AE00598984205DA5A
:105A300000EB800601EB460130390591501C0290C5
:105A4000029A1178A1F130000A28EED306940FF6DD
:105A5000F0101178FBF726FB20B10298401C029051
:105A6000401E00788DF81D009DF81D00682805D1A6
:105A70000299087868280CD1622206E06C2802BFDF
:105A8000029908786C2804D17122491C8DF81D20D8
:105A90000291029801780FF6A430FBF703FB80B95E
:105AA0000398401C0390012200980021C847064635
:105AB00000F0F6FD0028F3D1324669464846FFF76C
:105AC0004BFF00208DF81E0002980178253939D04F
:105AD0001C3900F09C80091F022940F2988013397C
:105AE00000F01083C91E1FD0891F00F09080891E0E
:105AF00000F08F84491E00F00583491E022940F200
:105B00008680091F00F0FE82491F3ED0491E0129F0
:105B100040F2F882091F35D0891E00F0F382C91EB9
:105B200000F0F08200F080BC224600F073BC2498A4
:105B3000002800F07A8416F1230F40F07684204686
:105B400000F082BC0398401C039001220098C847D3
:105B50000646252E0CD1B8F1000F48BF4FF00008C3
:105B60009DF81E0000283FF42AAF08F1010826E73F
:105B7000324669464846FFF7EFFE16F1010F40F046
:105B80005384AAE3012200F045BC9DF81C000028C4
:105B9000E1D19DF81D0062282DD0682811D06A2817
:105BA0001BD06C2801D0712817D0019951F8040B33
:105BB000019118B90FF68C2000F027BC0399016001
:105BC000C9E7019951F8040B019118B90FF6742037
:105BD00000F01BBC03990180BDE7019951F8040B4B
:105BE000019118B90FF65C2000F00FBC039AD3178F
:105BF000C0E90023AFE7019951F8040B019118B9EE
:105C00000FF6402000F001BC03990170A3E705984E
:105C10000028D8BF6FF00040049069464846FFF75F
:105C20008AFE00260AAF2B2818BF2D2807D18DF831
:105C3000280069464846FFF77EFE0DF1290700253A
:105C400030284FF00A0A16D169464846FFF773FE1E
:105C500040F02001C9B2782902D001252946ECE0A4
:105C600030203870797048466946FFF764FEBF1CE3
:105C70004FF0100AF2E740F02001CAB26E2A4CD170
:105C80006E2007F8010B69464846FFF754FE83462D
:105C90004BF02000C0B26128B24640F087816121FC
:105CA00007F8011B48466946FFF745FE83464BF05F
:105CB0002000C0B26E2840F0798169464846FFF75F
:105CC0003AFE282806D0024669464846FFF744FEB9
:105CD0006E2052E00498401E049004D50398401CA6
:105CE0000390A34604E069464846FFF71BFE83463F
:105CF000CDF820B0584600F0E7FC0028EAD1ABF11F
:105D000030000A28E6D308985F28E3D08346BBF129
:105D1000290F40F04B816E202FE0C9B2692940F075
:105D20009C80692007F8010B69464846FFF703FE8F
:105D300083464BF02000C0B26E28B24640F0368158
:105D40006E2107F8011B48466946FFF7F4FD8346BC
:105D50004BF02000C0B2662840F0288169464846D2
:105D6000FFF7E9FD40F02001C9B2692908D00246D9
:105D700069464846FFF7F0FD662007F8010B1BE176
:105D800003980499401C491E00290491039005D4EE
:105D9000009801220021C847834600E0A3464BF04B
:105DA0002000C0B26E2840F0018103980499401C85
:105DB000491E00290491039005D400980122002176
:105DC000C847834600E0A3464BF02000C0B26928D4
:105DD00040F0EC8003980499401C491E002904916E
:105DE000039005D4009801220021C847834600E0B3
:105DF000A3464BF02000C0B2742840F0D78003982F
:105E00000499401C491E00290491039005D4009870
:105E100001220021C847834600E0A3464BF0200042
:105E2000C0B2792840F0C280662107F8011BC3E0A8
:105E300069464846FFF776FD0121302808D10498CD
:105E4000401E0490F4D50398401C03902046F3E7CD
:105E50000D4611B1302107F8011B83462846002565
:105E600005E069464846FFF75DFD834601201BF1CA
:105E7000010F23D05FFA8BF2612AA8BFABF1570163
:105E80000ADA412AA8BFABF1370105DA303A0A2A0B
:105E900034BFABF13001FF21C9B251450ED2242DE0
:105EA000BABF07F801BB6D1C761C0498401E049015
:105EB000D7D50398401C0390A346D7E78DF8200060
:105EC0000995FBF71DFE406A01788B4510D107F854
:105ED00001BB03980499401C491E002904910390BA
:105EE00005D4009801220021C847834600E0A3465C
:105EF0000998E8B99DF8201005E069464846FFF783
:105F000011FD83460121BBF1300F09D10498761EA3
:105F1000401E0490F1D50398401C0390A346F1E77E
:105F2000002E8DF8201003D5302107F8011B761CB8
:105F30009DF82000099D05E069464846FFF7F2FC00
:105F4000834601201BF1010F23D05FFA8BF2612AF7
:105F5000A8BFABF157010ADA412AA8BFABF137015C
:105F600005DA303A0A2A34BFABF13001FF21C9B259
:105F700051450ED2242D08DB0498401E0490DBD539
:105F80000398401C0390A346DBE707F801BB6D1C98
:105F9000F2E7054650B14BF02000BAF10A0FC0B24B
:105FA00034D1652834D001E083460D465A4669460F
:105FB0004846FFF7D1FC0DB3002139709DF81C0055
:105FC00000287FF4C8ADBAF10A0F0B4674DC3246E4
:105FD0000AA800F073FC01228DF81E209DF81D20F8
:105FE000019B6C2A73D153F8042B0193002A6BD1C7
:105FF000DFF84404784400F5886006E20AA8874286
:1060000008BF1BF1010F40F00F8266E17028CDD16F
:1060100007F801BB0498401E049010D40398401C5C
:106020000390012200980021C8472B2818BF2D2873
:1060300011D107F8010B0498401E049004D5039871
:10604000401C0390204606E00398401C0390012268
:1060500000980021C847002104E069464846FFF740
:1060600061FC0121302808D10498401E0490F4D529
:106070000398401C03902046F3E70A001CBF30221F
:1060800007F8012B002504E069464846FFF74AFC63
:106090000121A0F130020A2A86D2082D08DB0498DB
:1060A000401E0490F0D50398401C03902046EFE773
:1060B00007F8010B6D1CF2E700220AA800F0FEFBB6
:1060C000B200FBF7D7F886E7C2E9000143E54C2AA6
:1060D0000AD153F8042B0193002AF5D1DFF85803B5
:1060E000784400F5557090E11E681A1D01922EB992
:1060F000DFF84403784400F5507086E100F09AFC24
:10610000306028E505980028CCBF401EDFF8280540
:1061100000280DF1200A04901BD40398401C039022
:10612000012200980021C8472B2818BF2D2814D120
:106130008DF820000DF1210A03980499401C491E96
:1061400000290491039007D4009801220021C84738
:1061500003E00399491C039120460021029A12781A
:10616000642A18BF752A0FD0692A08BF00260CD0F0
:106170006F2A08BF082608D0702A1CBF42F02002F0
:10618000782A02D1102600E00A2630282DD1049862
:106190000125401E0490039805D4401C0390012261
:1061A0000098C84702E0401C0390204640F02001C0
:1061B000C9B2782916D1002E18BF102E1DD104980F
:1061C0001026401E0490039807D4401C039001221F
:1061D00000980021C84700250FE0401C0390254689
:1061E00000274DE04EB9082607E0BEBB0A2635E081
:1061F00069464846FFF796FB0125302808D10498E8
:10620000401E0490F4D50398401C03902046F3E709
:106210002946CAB212B330220AF8012B1EE0412BE4
:10622000A8BFA0F1370306DAA3F130020A2A34BF6F
:10623000A0F13003FF23DBB2F2B293421ED21999D0
:106240008A4514D30498401E0490039812D4401C2D
:106250000390012200980021C847012110F1010F8D
:106260000CD0C3B2612BDADBA0F15703E3E70AF8E5
:10627000010BE7E7401C03900121204605460F462D
:106280002A4669464846FFF767FBFFB2F7B100218F
:106290008AF800109DF81C0000287FF45CAC02987E
:1062A0000078642818BF692869D0324608A800F031
:1062B000CBFC01228DF81E20029A1378702B10D18E
:1062C000019B53F8042B01934AB99CE008A882452E
:1062D00008BF15F1010F40F0A7802646A5E0106029
:1062E00039E49DF81D20622A39D0682A11D06A2A23
:1062F00025D06C2A06D0712A29D0742A18D07A2A7F
:106300000FD035E0019B53F8042B0193002AE6D10E
:1063100079E0019B53F8042B0193002A73D010807D
:1063200019E4019B53F8042B0193002AD7D16AE0AA
:10633000019B53F8042B0193002AD0D163E0019B09
:1063400053F8042B0193002A7FF4BEAE5BE0019B5F
:1063500053F8042B0193002A7FF4B6AE53E0019B5F
:1063600053F8042B0193002A4DD01070FFF7F3BBB4
:10637000019B53F8042B0193002AB0D143E032462D
:1063800008A800F0B5FC01228DF81E209DF81D2004
:10639000622AE4D0682ABCD06A2A1DD06C2A06D0B2
:1063A000712A21D0742A10D07A2A07D024E0019BC8
:1063B00053F8042B0193002A91D124E0019B53F858
:1063C000042B0193002A8AD11DE0019B53F8042B72
:1063D0000193002A83D116E0019B53F8042B01930B
:1063E000002A7FF471AE0EE0019B53F8042B019359
:1063F000002A7FF469AE06E0019B53F8042B019359
:10640000002A7FF46CAF00BF9DA0FAF765FE261A44
:1064100005E000226946484600F03CF80646002E9A
:106420003FF799ABFFF783BB0026B8F1000F7FF56C
:10643000D4AAB046FFF7D1BA7C1A0000CBCCCC0C62
:10644000686A6C747A4C00001BB0BDE8F08FC9B26A
:1064500008E003789942A4BF90F802C08C4515DA91
:10646000C01CD21E032A09D343782D2BF1D010F87B
:1064700001CB8C4518BF521EF4D107E042B110F891
:10648000013B8B4202D0521EF9D101E0012070473E
:10649000002070472DE9F04F92460027BAF1000F17
:1064A00083B080460E464FF0000B25D5B068411CE6
:1064B000B160084601785E2903BF401CB06010F847
:1064C000019DB946B56828785D280CBF681C284630
:1064D0005D21FAF7E7FD002800F0A680411B00913E
:1064E000B0600098032807DB821E2D21681CFAF794
:1064F0001DFE08B14FF0010B7069002805DCBAF1F0
:10650000000F14BF6FF0004001203061307F002881
:1065100001BF706850F8044B7060002C08D14FF038
:10652000FF3402487844001D11E000BF441A000007
:10653000307FA8B9F07F98B1716851F8040B716091
:10654000B0F1004FC0F007804FF0FF3444A0FAF7DD
:10655000C3FD201A6DE0B169884288BF0846B0616A
:10656000CDF80490CDF808B0DDF8009000E00227E7
:10657000F0683169401C491E00293161F06002D584
:106580004FF0FF3B38E0306801220021C0478346CE
:106590001BF1010F30D0BAF1000F0CDC1ED50298B0
:1065A000002801980AD000284A465946284612D0A9
:1065B000FFF74DFF09E000F073F806E000284A46B7
:1065C0005946284603D0FAF7B1FD38B114E0FAF77E
:1065D000ADFD88B102E0FFF73AFF68B1307F0028D7
:1065E000C5D1B06938B104F801BB0121B069B177F8
:1065F000401EB061BBE7012740465A463146FFF7CF
:10660000ABF9BAF1000F01D0022F09D0022F0FD041
:10661000F80702D41BF1010F06D14FF0FF3008E05C
:10662000307F28B9B06908B9002002E0002020704E
:10663000012003B0BDE8F08FFEFFFF7F63436E5B78
:10664000000000007363616E665F733A20626164EC
:1066500020256E20617267756D656E740000000004
:106660007363616E665F733A206261642025632CF8
:106670002025732C206F7220255B2073697A6500BA
:106680007363616E665F733A2062616420696E7441
:106690006567657220617267756D656E74000000D4
:1066A00010B50446FBF72AFA01462046096ABDE800
:1066B0001040084710B50446FBF720FA0146204673
:1066C000896ABDE81040084710B50446FBF716FA82
:1066D000014620460969BDE810400847F8B52DED90
:1066E000048B140082B041EC180B1D4600F0DA80D8
:1066F00031F0004108BF002800F0D48051EC180BA5
:106700004A00521512F1010F02D1080300F0CA80AD
:10671000002C9FED689B57D56442654F7F4407F579
:10672000C87708260CE0E00707D5D7E9002351EC2D
:10673000190BFBF7EFF841EC190B64080837761ECC
:10674000002C18BF002EEED16A4651EC180BFAF758
:1067500025FD009E53EC192BFAF798FF3246FAF705
:1067600089FD41EC180B31F0004108BF002800F012
:10677000828051EC180B4A00521512F1010F01D121
:10678000080378D0002C76D06A4651EC180BFAF743
:1067900005FD009E994A9A4BFBF7BCF83246FAF782
:1067A00069FD41EC180B31F0004108BF002862D0B0
:1067B00051EC180B4A00521512F1010F01D10803D8
:1067C00059D0641EE0D156E055DD394F7F4407F1C2
:1067D000E0070826E00707D5D7E9002351EC190B9D
:1067E000FBF798F841EC190B64100837761E002C63
:1067F00001DD002EEED16A4651EC180BFAF7CEFC03
:106800002646009C53EC192BFBF784F82246FAF736
:1068100031FD41EC180B31F0004108BF00282AD0AF
:1068200051EC180B4A00521512F1010F01D1080367
:1068300021D0002E1FDD6A4651EC180BFAF7AEFC92
:10684000009C704A784BFBF765F82246FAF712FD78
:1068500041EC180B31F0004108BF00280BD051EC7F
:10686000180B4A00521512F1010F01D1080302D092
:10687000761E002EDFDC51EC180B31F0004108BF12
:10688000002808D051EC180B4A00521512F1010FE4
:1068900008D1080306D1AFF300801DB1286840F08D
:1068A0000100286002B051EC180BBDEC048BF4BD64
:1068B00010150000000000000000F03F2DE9F14D30
:1068C00081B00C462DED028B84B093465FEA030A3B
:1068D0001CBF0020CAF80000079D07A800F00BFAB3
:1068E000C11020F00800012801F0010832D1022077
:1068F000009001AB07992246284600F08DFA04006B
:1069000008BF9FED4A0B1ED00298FAF77DFD022CBE
:1069100041EC100B17DB03AF661E9FED3B8B51EC78
:10692000100B53EC182BFAF7F5FF044657F8040B3D
:106930000D46FAF769FD22462B46FAF777FD761EDB
:1069400041EC100BEBD1019800EB0B02534651ECDC
:10695000100B33E0022836D1009001AB0799224694
:10696000284600F035FB040008BF9FED300B1ED019
:106970000298FAF749FD022C41EC100B17DB03AF2C
:10698000661E9FED238B51EC100B53EC182BFAF77E
:10699000C1FF044657F8040B0D46FAF735FD2246B1
:1069A0002B46FAF743FD761E41EC100BEBD1019A12
:1069B00051EC100BFAF75EFC53465A46FFF78EFE79
:1069C00041EC100B0AE0032808BF9FED130B05D024
:1069D00004280CBF9FED120B9FED140BB8F1000FB4
:1069E00005D051EC100B81F0004141EC100B04B0CC
:1069F00051EC100BBDEC028BBDE8FC8D436FAC6419
:106A00002806C80A3CBF737F0000000065CDCD4159
:106A1000000000000000B041000000000000F07F16
:106A2000FFFFFFFFFFFFFF7FDD4F15750000000038
:106A30000000000001F000428B1AA3F16051B1F593
:106A4000801F0ADBB1F17F6F1FD242EAC102C10091
:106A500071F1004142EB507070470B15C3F109030F
:106A6000212B10D2890241EA90518002012849412C
:106A700041F0004121FA03F0C3F12003994071F184
:106A8000004150417047100070476FF0000013EB59
:106A9000103F5CBF000E42EAC05070472DE9FC4F2A
:106AA00085B00C4693460BB100221A6002908246D4
:106AB00001E00AF1010A9AF80000FFF7F1FD002851
:106AC000F7D19AF800002D2818BF2B2807BF1AF815
:106AD000010B8DF800002B218DF80010BBF1000F89
:106AE000019405D4BBF1010F02D0BBF1250F04DBEB
:106AF000002C72D0029820606FE0BBF1000F0DDD1A
:106B0000BBF1100F04BF9AF80000302802BF9AF8BA
:106B1000010040F02000782814D10EE09AF800001F
:106B2000302818BF4FF00A0B0CD19AF8010040F042
:106B30002000782804D14FF0100B0AF1020A01E07E
:106B40004FF0080BCDF810A001E00AF1010A9AF805
:106B500000003028F9D0094878442030002428303B
:106B600000260027CDF80CA00025A0468DF80100D6
:106B7000DFF80890F94409F1040919E0C411000094
:106B800001469DF80100081A5FFA80F85846A0FBFC
:106B900006234FEAEB7100FB073301FB0633344653
:106BA00000213D4612EB080643EB01070AF1010AFA
:106BB0009AF80000FFF77EFD01465A4609F12800C9
:106BC000FAF7B4FA0028DBD1049951455A4607D1A7
:106BD000019810B10199029808600020002130E06E
:106BE000039919F80200AAEB0101091A00291BD424
:106BF00010DC0023B6EB080067EB03018F4209D3DA
:106C000001D8864206D3D317FAF780FFA94208BFFE
:106C1000A04209D0AFF30080069808B101210160BD
:106C20004FF0FF36374606E09DF800002D2802D1D0
:106C3000764267EB4707019808B1C0F800A03046DC
:106C4000394607B0BDE8F08F00BF002326E70000FB
:106C50002DE9F8430D0091461E4608BF6D4680465B
:106C6000444600E0641C2078FFF71AFD0028F9D1A3
:106C700027782D2F18BF2B2F05D114F8010FFFF700
:106C80000FFD08B109E02B2733464A462946204626
:106C9000FFF704FF2A68944205D1C5F80080002060
:106CA0000021BDE8F4832B2F05D14FF0004399421A
:106CB00009D2BDE8F4832D2FFBD1B1F1004F12D3DF
:106CC00001D801280FD3AFF300800EB1012030604E
:106CD0002D2F19BF4FF0FF306FF0004100204FF013
:106CE0000041BDE8F483404261EB4101BDE8F4831B
:106CF00000BF0023ACE72DE9F84305460C462E689B
:106D0000002700E0761C3078FFF7CAFC0028F9D194
:106D100030782D280CBF08272B2800D1761C30781E
:106D200040F020016E2927D1707840F020006128C2
:106D300002BFB07840F020006E2802D02E680027F5
:106D400046E0F61CB046042798F8000028283FD1FA
:106D500018F8019F4846FFF7B7FC0028F8D1A9F1C1
:106D600030000A28F4D398F800005F28F0D02928D2
:106D70002ED108F101062BE069292CD1707840F062
:106D800020006E2802BFB07840F02000662802D0B4
:106D90002E6800271CE016F8030F40F0200047F093
:106DA0000307692802BF707840F020006E280FD1D9
:106DB000B07840F02000692802BFF07840F0200051
:106DC000742805D1307940F02000792808BF761D5D
:106DD000F4B126601CE0302802BF707840F020003B
:106DE000782813D1B01C01782E2908BF401C0078E8
:106DF000A0F16101062921BFA0F14102062A303825
:106E00000A2803D2B61C47F0020701E047F0010749
:106E10002E603846BDE8F2832DE9F14F8CB04FF07B
:106E20000008169D05EBC5059246C3462D2DC8BF2B
:106E30002D25C3F800B0C3F804B0D94602E0491CC0
:106E40004FF0010908783028F9D0002411E01868C3
:106E5000401C18600A78302A08D04FF0010805E07D
:106E6000AC42F4DA30380DF80400641C491C4FF0D1
:106E700001090878A0F130020A2AF1D30F461E4614
:106E8000FAF73EFE406A39780278914208BF7F1CCB
:106E9000002C48460ED1397830290BD13068401E7D
:106EA00030607F1C0120F6E7302918BF4FF0010841
:106EB0007F1C01203978A1F130020A2A0AD2AC42A3
:106EC000F2DAA1F130000DF80400641C3268521EA1
:106ED0003260EDE7B8F1000F0DD00DF1FF314A5DE2
:106EE000521C4A5507E00DF1FF32115D49B9326875
:106EF000521C3260641E002CF5DC04BF8DF800B01B
:106F00000124002856D0092394FBF3F3C4F10909A6
:106F100003EBC3034B44092193FBF1F1002201EB86
:106F2000C101591A1AD04FF0010B17E056F82B1077
:106F300001EB810105EB410146F82B100CE0092122
:106F400093FBF1F101EBC1011DF80250591AEDD18B
:106F50000BF1010B46F82B505B1C521CA242EEDBDE
:106F6000397841F02001652924D1394617F8012FDD
:106F70002B2A16BF2D2A17F8014B2B2400220023A1
:106F8000124D08E0AB4204DA03EB83020CEB420340
:106F9000303B7F1C012297F800C0ACF1300EBEF1EF
:106FA0000A0FEFD32D2C08BF5B4234681B193360E6
:106FB00002B90F46BAF1000F03D000B90C9FCAF80E
:106FC000007058460DB0BDE8F08F00BF00E1F50538
:106FD0002DE9F14F8CB09146DDF85880C8EBC80818
:106FE0004FF0000AB8F1230FC8BF4FF02308C3F8D1
:106FF00000A0C3F804A0002701E0491C012708787D
:107000003028FAD068A201925FF000046CA20092CE
:107010000DF1080B0D461E460EE03068401C306036
:1070200008E0A045F9DB019A0099801A085C0BF88A
:107030000400641C6D1C012795F800105AA016224C
:10704000FAF774F80028ECD1FAF75AFD406A29786B
:107050000278914208BF6D1CB4B92878302813D14A
:107060003168491E31606D1C0127F6E7A04509DB38
:10707000019A0099801A085C0BF80400641C3168BE
:10708000491E31606D1C01272978162246A0FAF7A7
:107090004DF80028EAD1A04517DA1BF80810072997
:1070A00006DD0DF1070111F80820521C01F8082037
:1070B00044463268521C326007E00DF10702115D50
:1070C00049B93268521C3260641E002CF5DC04BFE2
:1070D0008DF808A0012431688900002F316055D057
:1070E000072394FBF3F3C4F1070BC3EBC3035B4427
:1070F000072193FBF1F10022C1EBC101591A19D00C
:107100004FF0010A16E056F82A100BEB011046F872
:107110002A000DE0072102A893FBF1F1C1EBC101A8
:1071200010F802B0591AEED10AF1010A46F82AB055
:107130005B1C521CA242EDDB297841F02001702932
:1071400024D1294615F8012F2B2A16BF2D2A15F810
:10715000014B2B2400220023124808E0834204DA6A
:1071600003EB83020CEB4203303B6D1C012295F8CC
:1071700000C0ACF1300EBEF10A0FEFD32D2C08BFCA
:107180005B4234681B19336002B90D46B9F1000F38
:1071900003D007B90C9DC9F8005050460DB0BDE8AA
:1071A000F08F000000E1F5053031323334353637E9
:1071B0003839616263646566414243444546000074
:1071C000000102030405060708090A0B0C0D0E0F47
:1071D0000A0B0C0D0E0F0000100000004F4B0D0AA3
:1071E000000000000000000000000000000000009F
:1071F000000000000000000000000000000000008F
:10720000000000000000000000000000000000007E
:10721000000000000000000000000000000000006E
:10722000000000000000000000000000000000005E
:10723000000000000000000000000000000000004E
:10724000080000003E0000000000000000000000F8
:10725000000000000000000000000000000000002E
:10726000000000000000000000000000000000001E
:10727000000000000000000000000000000000000E
:1072800000000000000000000000000000000000FE
:1072900000000000000000000000000000000000EE
:1072A0000000000000000000004000004349505270
:1072B0005847455400000000000000000000000096
:1072C00000000000000000000000000000000000BE
:1072D00000000000000000000000000000000000AE
:1072E000000000000000000000000000000000009E
:1072F000000000000000000000000000000000008E
:10730000000000000000000000000000000000007D
:107310000000040043495053454E44000000000063
:10732000000000000000000000000000000000005D
:10733000000000000000000000000000000000004D
:10734000000000000000000000000000000000003D
:10735000000000000000000000000000000000002D
:10736000000000000000000000000000000000001D
:10737000000000000000000000000200504F5745D0
:1073800052454420444F574E0D0A000000000000B3
:1073900000000000000000000000000000000000ED
:1073A00000000000000000000000000000000000DD
:1073B00000000000000000000000000000000000CD
:1073C00000000000000000000000000000000000BD
:1073D00000000000000000000000000000000000AD
:1073E000000009005244590D0A000000000000008E
:1073F000000000000000000000000000000000008D
:10740000000000000000000000000000000000007C
:10741000000000000000000000000000000000006C
:10742000000000000000000000000000000000005C
:10743000000000000000000000000000000000004C
:10744000000000000000000080000000636C6F730B
:107450006564220000000000000000000000000041
:10746000000000000000000000000000000000001C
:10747000000000000000000000000000000000000C
:1074800000000000000000000000000000000000FC
:1074900000000000000000000000000000000000EC
:1074A00000000000000000000000000000000000DC
:1074B0000001000043495052584745543A53554340
:1074C000434553530000000000000000000000008E
:1074D00000000000000000000000000000000000AC
:1074E000000000000000000000000000000000009C
:1074F000000000000000000000000000000000008C
:10750000000000000000000000000000000000007B
:10751000000000000000000000020000696E636FC0
:107520006D696E672066756C6C22000000000000BB
:10753000000000000000000000000000000000004B
:10754000000000000000000000000000000000003B
:10755000000000000000000000000000000000002B
:10756000000000000000000000000000000000001B
:10757000000000000000000000000000000000000B
:1075800000040000696E636F6D696E672200000081
:1075900000000000000000000000000000000000EB
:1075A00000000000000000000000000000000000DB
:1075B00000000000000000000000000000000000CB
:1075C00000000000000000000000000000000000BB
:1075D00000000000000000000000000000000000AB
:1075E00000000000000000000008000070647064EB
:1075F00065616374220000000000000000000000CC
:10760000000000000000000000000000000000007A
:10761000000000000000000000000000000000006A
:10762000000000000000000000000000000000005A
:10763000000000000000000000000000000000004A
:10764000000000000000000000000000000000003A
:10765000001000002B4D444E534749503A000000A3
:10766000000000000000000000000000000000001A
:10767000000000000000000000000000000000000A
:1076800000000000000000000000000000000000FA
:1076900000000000000000000000000000000000EA
:1076A00000000000000000000000000000000000DA
:1076B0000000000000000000400000004552524F52
:1076C000520D0A0000000000000000000000000051
:1076D00000000000000000000000000000000000AA
:1076E000000000000000000000000000000000009A
:1076F000000000000000000000000000000000008A
:107700000000000000000000000000000000000079
:107710000000000000000000000000000000000069
:1077200000800000434D45204552524F523A000020
:107730000000000000000000000000000000000049
:107740000000000000000000000000000000000039
:107750000000000000000000000000000000000029
:107760000000000000000000000000000000000019
:107770000000000000000000000000000000000009
:107780000000000000000000002000004552524FA1
:10779000520D0A0000000000000000000000000080
:1077A00000000000000000000000000000000000D9
:1077B00000000000000000000000000000000000C9
:1077C00000000000000000000000000000000000B9
:1077D00000000000000000000000000000000000A9
:1077E0000000000000000000000000000000000099
:1077F000020000004F4B0D0A0000000000000000D6
:107800000000000000000000000000000000000078
:107810000000000000000000000000000000000068
:107820000000000000000000000000000000000058
:107830000000000000000000000000000000000048
:107840000000000000000000000000000000000038
:107850000000000000000000200000004F50454ED6
:107860003A000000000000000000000000000000DE
:107870000000000000000000000000000000000008
:1078800000000000000000000000000000000000F8
:1078900000000000000000000000000000000000E8
:1078A00000000000000000000000000000000000D8
:1078B00000000000000000000000000000000000C8
:1078C0000400000072656164790D0A000000000088
:1078D00000000000000000000000000000000000A8
:1078E0000000000000000000000000000000000098
:1078F0000000000000000000000000000000000088
:107900000000000000000000000000000000000077
:107910000000000000000000000000000000000067
:107920000000000000000000000008000D0A0D0A21
:107930004F4B0000000000000000000000000000AD
:107940000000000000000000000000000000000037
:107950000000000000000000000000000000000027
:107960000000000000000000000000000000000017
:107970000000000000000000000000000000000007
:1079800000000000000000000000000000000000F7
:10799000100008000D0A0D0A0000000000000000A1
:1079A00000000000000000000000000000000000D7
:1079B00000000000000000000000000000000000C7
:1079C00000000000000000000000000000000000B7
:1079D00000000000000000000000000000000000A7
:1079E0000000000000000000000000000000000097
:1079F0000000000000000000100009002B51504959
:107A00004E473A2000000000000000000000000087
:107A10000000000000000000000000000000000066
:107A20000000000000000000000000000000000056
:107A30000000000000000000000000000000000046
:107A40000000000000000000000000000000000036
:107A50000000000000000000000000000000000026
:107A6000010000000D0A00000000000000000000FE
:107A70000000000000000000000000000000000006
:107A800000000000000000000000000000000000F6
:107A900000000000000000000000000000000000E6
:107AA00000000000000000000000000000000000D6
:107AB00000000000000000000000000000000000C6
:107AC0000000000000000000537563636573736677
:107AD000756C20496E697469616C697A6174696F4B
:107AE0006E206F6620746865204D6F64756C650D3F
:107AF0000A0D0A005369676E616C205175616C69EB
:107B00007479204C6576656C2025642064426D2074
:107B10002847534D20466F726D61743A20256C647E
:107B2000290D0A005369676E616C205175616C699B
:107B30007479204C6576656C206E6F742064657472
:107B400065637461626C650D0A0000000D0A203ED9
:107B50003E3E204D6F64756C652052656769737495
:107B6000726174696F6E20537563636573736675B4
:107B70006C0D0A0D0A0000000D0A203E3E3E204D0D
:107B80006F64756C6520526567697374726174699E
:107B90006F6E20547279696E670D0A0D0A0000003D
:107BA0000D0A203E3E3E204D6F64756C6520526587
:107BB00067697374726174696F6E2044656E69657C
:107BC000640D0A0D0A0000000D0A203E3E3E204DC5
:107BD0006F64756C6520526567697374726174694E
:107BE0006F6E204661696C65640D0A0D0A00000025
:107BF0000D0A203E3E3E204D6F64756C6520415459
:107C000020436F6D6D756E69636174696F6E204599
:107C100072726F7220776974682074686520446599
:107C2000766963650D0A0000203E3E3E204465767D
:107C3000696365206D696768742062652064697393
:107C4000636F6E6E6563746564206F722077726F08
:107C50006E676C7920636F6E6E65637465640D0A80
:107C60000D0A0000203E3E3E20506C656173652089
:107C7000636865636B206966207468652053494DAD
:107C800020697320696E73657274656420616E6427
:107C90002076616C69642C20696620637265646576
:107CA0006E7469616C7320617265206F6B2C206546
:107CB00074632E0D0A0D0A000D4661696C6564201F
:107CC000746F2067657420746865206375727265CF
:107CD0006E742063656C6C756C6172206F70657278
:107CE00061746F72206E616D650D0A0D0A000000EF
:107CF00000002115110E0D0C0B0B0A0A09090909C8
:107D000009080808080808080707070707070707FA
:107D100007070707070000003031323334353637A4
:107D200038396162636465666768696A6B6C6D6E39
:107D30006F707172737475767778797A00000000CD
:107D400000004129211C19171615141312121111C4
:107D5000111010100F0F0F0F0E0E0E0E0E0E0E0D37
:107D60000D0D0D0D0D000000303132333435363736
:107D700038396162636465666768696A6B6C6D6EE9
:107D80006F707172737475767778797A000000007D
:107D90004661696C20746F2041542053594E432C26
:107DA000206166746572207365766572616C20610E
:107DB0007474656D7074730D0A000000000000009B
:107DC00000000000000024400000000000005940B6
:107DD000000000000088C3400000000084D79741E5
:107DE0000080E03779C34143176E05B5B5B89346B7
:107DF000F5F93FE9034F384D321D30F94877825A83
:107E00003CBF737FDD4F157580B50D497944303126
:107E10000C4A7A442E32914203D00B49AFF30080D2
:107E200002BD8DF80000012269460120FAF7BEFF6D
:107E3000012802D19DF8000002BD4FF0FF3002BDC5
:107E4000C081FFF7BC81FFF79000002030B400250F
:107E500012E050F8042BD30744BF4A44521E091FB6
:107E6000042942F8045BFAD213468C0744BF1580FC
:107E70009B1CC90748BF1D7050F8041B0029E8D19E
:107E800030BC70475369676E616C206973206E6FF8
:107E900074206B6E6F776E206F72206E6F7420642B
:107EA000657465637461626C65207965742E2E2E2D
:107EB000200000007363616E665F733A2062616444
:107EC00020666C6F6174696E672D706F696E7420C7
:107ED000617267756D656E740000000010B507492A
:107EE00079441831064C7C44163404E00A68081DB5
:107EF000114488470146A142F8D110BD0801000095
:107F00002401000041542B5149435347503D2564FF
:107F10002C312C222573222C222573222C2225730E
:107F2000222C25640D0A0000202D2D2D20515545B1
:107F30004354454C204547393120506F77657220B6
:107F40005570202D2D2D0D0A00000000202D2D2D07
:107F5000205155454354454C2045473931205368FD
:107F6000757420446F776E202D2D2D200D0A000092
:107F70007363616E665F733A206261642025632CCF
:107F80002025732C206F7220255B20617267756D30
:107F9000656E7400FEE7FEE7FEE7FEE7FEE770476A
:107FA0007047704700F008B80148F9F727BF000094
:107FB000740B002000F008B802494A68087882185B
:107FC0004A607047000000200349C8680A6882437D
:107FD0000A60486000F002B8001D0C4270470000C3
:107FE0004EF68851CEF20001086840F47000086037
:107FF000BFF34F8FBFF36F8F4FF00170E1EE100AA8
:108000007047000049FEFFFFB80B0000D8000020B9
:10801000000000001390FFFF9C010000B40000006E
:108020000000002000F00DF8002801D0FFF756FFF7
:10803000AFF300800020AFF30080FBF7FFFA00F001
:1080400002F80120704700F001B8000007463846EA
:10805000F9F7E4FDFBE700000548014603B4684674
:1080600080F30988AFF30080FFF7BAFFFFF7DAFF6C
:10807000A5EDF5FE38B504460D462846FFF7C4FECB
:10808000A84218BF0024204632BD000001488047A6
:1080900001480047B546000859800008000000006C
:1080A00001020304FFF7FEBFFFF7FEBFFFF7FEBFAD
:1080B000FFF7FEBFFFF7FEBFFFF7FEBFFFF7FEBFF4
:1080C000FFF7FEBFFFF7FEBFFFF7FEBFFFF7FEBFE4
:1080D000FFF7FEBFFFF7FEBFFFF7FEBFFFF7FEBFD4
:1080E000FFF7FEBFFFF7FEBFFFF7FEBFFFF7FEBFC4
:1080F000FFF7FEBFFFF7FEBFFFF7FEBFFFF7FEBFB4
:10810000FFF7FEBFFFF7FEBFFFF7FEBFFFF7FEBFA3
:10811000FFF7FEBFFFF7FEBFFFF7FEBFFFF7FEBF93
:10812000FFF7FEBFFFF7FEBFFFF7FEBFFFF7FEBF83
:10813000FFF7FEBFFFF7FEBFFFF7FEBFFFF7FEBF73
:10814000FFF7FEBFFFF7FEBFFFF7FEBFFFF7FEBF63
:10815000FFF7FEBFFFF7FEBFFFF7FEBFFFF7FEBF53
:10816000FFF7FEBFFFF7FEBFFFF7FEBFFFF7FEBF43
:10817000FFF7FEBFFFF7FEBFFFF7FEBFFFF7FEBF33
:10818000FFF7FEBFFFF7FEBFFFF7FEBFFFF7FEBF23
:10819000FFF7FEBFFFF7FEBFFFF7FEBFFFF7FEBF13
:1081A000FFF7FEBFFFF7FEBFFFF7FEBFFFF7FEBF03
:1081B000FFF7FEBF43010001221008F0050724F479
:1081C00000D21800080452FF01E32A14142004000E
:1081D000008A1600084C114822204B2002C71A00C2
:1081E000080852C10812DD0812C50452F110E1015D
:1081F0006188100702040101080C0020580452088D
:0E82000004211B610812D46052C064F10B010E
:040000050800805916
:00000001FF
